:100000000C941E060C94D3280C9400290C944606DC
:100010000C9446060C9446060C9446060C94460630
:100020000C9446060C9446060C941B130C9446063E
:100030000C9446060C9446060C9446060C94460610
:100040000C942D290C9446060C941B2D0C945E2DBB
:100050000C9446060C9446060C9446060C944606F0
:100060000C9446060C9446062419861965196819DD
:100070006B196E1971197419771986198019B81AC4
:10008000BA1ABA1AB81ABA1ABA1ABA1ABA1ABA1AD2
:10009000BA1ABA1ABA1ABA1ABA1ABA1ABA1ABA1AC0
:1000A0003E1ABA1ABA1ABA1ABA1ABA1AAF19BA1A38
:1000B000BA1ABA1ABA1ABA1ABA1ABA1ABA1ABA1AA0
:1000C000BA1ABA1ABA1ABA1ABA1ABA1A4A1A4A1A70
:1000D0004A1A4A1A4A1A4A1A4A1A4A1A4A1ABA1A90
:1000E000BA1ABA1ABA1ABA1ABA1AAF19491A491A5E
:1000F000491A491ABA1A571A5D1A631A691A6F1AF5
:10010000751A7B1A811A8B1A951A9F1AA91AF01957
:10011000B219BA1ABA1ABA1ABA1A3E1ABA1ABA1AC4
:10012000BA1ABA1ABA1ABA1ABA1ABA1A481A481A13
:10013000481A481ABA1A571A5D1A631A691A6F1AB6
:10014000751A7B1A811A8B1A951A9F1AA91AF01917
:10015000B219BA1ABA1ABA1ABA1A3E1AED1AED1A1E
:10016000ED1AED1AED1AED1AED1AED1AED1AED1A57
:10017000ED1AED1AED1A041C041C041C041C041CCA
:10018000041C321B3C1B461B501BAE1BB81BC71B61
:10019000D81B601D751D811D8A1D991DBE1DC71DA3
:1001A000101ED91D24212A21302137214521672104
:1001B0008521456E746572206D656E752E2E2E003C
:1001C000546F67676C6564206D6963726F50504D42
:1001D00000546F67676C656420696E76657274653C
:1001E000642050504D2100546F67676C6564205443
:1001F00058206D7574696E672100546F67676C6570
:10020000642074656C656D65747279210050726F3D
:10021000746F636F6C206572726F72207769746897
:100220002052580054696D656F7574207768656E4B
:1002300020636F6E6E656374696E6720746F205201
:100240005800507265737320616E79206B65792058
:10025000746F2063616E63656C00436F6E6E6563DF
:1002600074696E6720746F2052582C20706F776508
:100270007220757020746865205258202877697440
:10028000682062696E6420706C7567206966206EF4
:100290006F74207573696E6720616C776179732064
:1002A00062696E642900546F67676C656420276912
:1002B0006D6D656469617465206F75747075742700
:1002C00000546F67676C65642027736C61766520E6
:1002D0006D6F64652700546F67676C6564202761E4
:1002E0006C776179732062696E642700546F676769
:1002F0006C65642050504D206368616E6E656C20A3
:100300006C696D69740053657420525353492069B8
:100310006E6A656374696F6E206368616E6E656C8A
:100320002028303D3D64697361626C652900536526
:10033000742050504D206D696E696D756D20737914
:100340006E630053657420626561636F6E20696E31
:1003500074657276616C0053657420626561636FC9
:100360006E2064656C617900536574206265616319
:100370006F6E206672657175656E637920696E2097
:10038000487A3A20303D64697361626C652C205074
:10039000783D504D52206368616E6E656C20782CFC
:1003A0002046783D465253206368616E6E656C202E
:1003B00078005365742050574D2073746F7020641B
:1003C000656C61792028302064697361626C6564B2
:1003D0002C20312D323535203D3D20302E317320FB
:1003E0002D2035306D696E29005365742050504DB5
:1003F0002073746F702064656C61792028302064EC
:10040000697361626C65642C20312D323535203D75
:100410003D20302E3173202D2035306D696E29003E
:10042000536574206661696C736166652064656CF0
:1004300061792028302064697361626C65642C20C6
:10044000312D323535203D3D20302E3173202D2089
:1004500035306D696E29002A2A2A2A2A2A2A2A2A50
:100460002A2A2A2A2A2A2A2A2A2A2A2A2A2A2A2AEC
:100470002A2A2A2A0052582041636B6564202D20C5
:1004800072657665727420737563636573736675E0
:100490006C21002A2A2A2A2A2A2A2A2A2A2A2A2AAD
:1004A0002A2A2A2A2A2A2A2A2A2A2A2A2A2A2A2AAC
:1004B000002A2A2A2A2A2A2A2A2A2A2A2A2A2A2AC6
:1004C0002A2A2A2A2A2A2A2A2A2A2A2A2A2A00528E
:1004D000582041636B6564202D20757064617465DC
:1004E000207375636365737366756C21002A2A2A0D
:1004F0002A2A2A2A2A2A2A2A2A2A2A2A2A2A2A2A5C
:100500002A2A2A2A2A2A2A2A2A2A0056616C696457
:100510002063686F69636573206172653A205B319F
:100520005D2D5B31365D20286368616E6E656C20E1
:10053000312D31362900536574206F7574707574D0
:1005400020666F7220706F727420005B585D2061AE
:10055000626F7274206368616E67657320616E6498
:10056000206578697420525820636F6E6669670051
:100570005B535D20736176652073657474696E6783
:100580007320746F205258005B525D20726576654F
:1005900072742052582073657474696E6773207486
:1005A0006F2064656661756C747300557365206EA9
:1005B000756D62657273205B312D445D20746F2010
:1005C0006564697420706F727473205B452D515D92
:1005D00020666F722073657474696E677300202DD6
:1005E00020726563656976657220636F6E66696700
:1005F000757261746F722C20727820737720000AF4
:100600000A6F70656E4C52536E67200053657420FC
:1006100073657269616C2062617564726174653AB8
:10062000200056616C69642063686F696365733A82
:100630002031202D20342B34202F2032202D203823
:10064000202F2033202D20382B34202F2034202D14
:10065000203132202F2035202D2031322B34202FF5
:100660002036202D20313600536574204368616E9A
:100670006E656C20636F6E6669673A20005365741F
:100680002044617461726174652028302D32293AEA
:10069000200053657420486F70206368616E6E653A
:1006A0006C7320286D61782032342C207365706162
:1006B000726174656420627920636F6D6D61732966
:1006C0002076616C69642076616C75657320312DCC
:1006D0003235353A2000536574206368616E6E656B
:1006E0006C2073706163696E6720287831306B48C5
:1006F0007A293A200053657420524620706F77653E
:10070000722028302D37293A200053657420524634
:10071000206D6167696320286865782920652E67E8
:100720002E20307844454144463030443A2000532E
:1007300065742062617365206672657175656E63AC
:10074000792028696E20487A293A20005B5A5D207A
:10075000656E746572207265636569766572206383
:100760006F6E66696775726174696F6E2075746902
:100770006C79005B465D20646973706C61792061FF
:10078000637475616C206672657175656E63696509
:10079000732075736564005B525D2063616C6375E3
:1007A0006C6174652072616E646F6D206B65792079
:1007B000616E6420686F70206C697374005B495DC2
:1007C000207265696E697469616C697A6520736508
:1007D0007474696E677320746F20736B65746368DB
:1007E0002064656661756C7473005B585D2072658A
:1007F00076657274206368616E67657320616E64EC
:100800002065786974206D656E75005B535D20739B
:100810006176652073657474696E677320746F20E8
:10082000454550524F4D20616E64206578697420B3
:100830006D656E7500557365206E756D62657273BA
:10084000205B302D395D20746F20656469742070E1
:100850006172616D657465727300202D2053797328
:1008600074656D20636F6E66696775726174696F18
:100870006E000A0A6F70656E4C52536E672000510D
:1008800029204F7574707574206265666F726520DB
:100890006C696E6B20283D465329203A2000502970
:1008A00020536C617665206D6F64652028657870D3
:1008B0006572696D656E74616C293A20004F29205C
:1008C00054696D65642042494E44206174207374FC
:1008D000617274757020203A20004E292050504DCE
:1008E000206F7574707574206C696D69746564200F
:1008F000202020203A200044495341424C454400E6
:100900004D292050504D205253534920746F20637D
:1009100068616E6E656C202020203A20004C2920F2
:1009200050504D206D696E696D756D2073796E63E1
:10093000202875732920203A200044495341424C15
:100940004544004B29204661696C736166652062ED
:100950006561636F6E20696E74762E2028312D32AA
:10096000353573293A20004A29204661696C736144
:10097000666520626561636F6E2064656C617920D5
:1009800028302D323535203D3E20313073202D204A
:100990003135306D696E293A200049292046616958
:1009A0006C7361666520626561636F6E206672714B
:1009B0002E203A200048292050574D2073746F7024
:1009C0002064656C6179202020202020203A2000BE
:1009D00047292050504D2073746F702064656C61FE
:1009E00079202020202020203A200046292046611E
:1009F000696C736166652064656C617920202020D4
:100A00002020203A200050574D206368616E6E65AB
:100A10006C200066756E6374696F6E3A2000292041
:100A2000706F72742000506F776572546F776572C3
:100A300000445446205548462033322D62697420C4
:100A400031306368004F70656E4C52536E67525878
:100A5000206D696E6920342F36636800466C7974A6
:100A6000726F6E2F4F72616E6765525820554846FF
:100A70002038636800525820747970653A20004429
:100A8000697361626C656400487A00203D3D200016
:100A900043616C63756C61746564207061636B6540
:100AA0007420696E74657276616C3A200042292068
:100AB0004D6963726F202868616C66292050504D23
:100AC000202020203A00412920496E766572746505
:100AD000642050504D20696E20202020203A0030A4
:100AE00029204D7574652062757A7A657220286DAB
:100AF0006F73746C79293A003929205365726961E2
:100B00006C2062617564726174653A00736D617224
:100B100074506F7274004672536B79005472616E38
:100B200073706172656E740044697361626C6564B0
:100B30000038292054656C656D657472793A2020FF
:100B40002020202020003729204368616E6E656CCC
:100B500020636F6E6669673A202000362920446161
:100B60007461726174652028302D32293A2020206A
:100B700000352920486F70206368616E6E656C7364
:100B80003A2020202020003429204368616E6E65C1
:100B90006C2073706163696E673A202000332920EE
:100BA000524620706F7765722028302D37293A2001
:100BB0002020003229205246206D616769633A2067
:100BC0002020202020202020003129204261736530
:100BD000206672657175656E63793A202020000089
:100BE00000000700020100000304060000000000EE
:100BF00000000001020408102040800102040810D7
:100C00002001020408102004040404040404040263
:100C10000202020202030303030303000000002395
:100C2000002600290000000000250028002B0000FD
:100C3000000000240027002A00004C2E11241FBEB3
:100C4000CFEFD8E0DEBFCDBF13E0A0E0B1E0E6EA31
:100C5000F2E602C005900D92A83CB107D9F716E064
:100C6000A8ECB3E001C01D92A239B107E1F71CE086
:100C7000CCE3DCE004C02297FE010E94552FCA336A
:100C8000D107C9F70E94882E0C9451310C940000B2
:100C900080917705813019F482E080937705809107
:100CA0007705833019F484E0809377050895A8953B
:100CB0000895DC01ED91FC910190F081E02D099502
:100CC00008952091780530917905382748E0C901C9
:100CD000880F991F37FF06C09C0151E2252750E17C
:100CE000352701C09C01415091F73093790520933D
:100CF0007805089588E380937A0580E092ECA1E07E
:100D0000B0E080937B0590937C05A0937D05B09324
:100D10007E0587E08093870580EC92E9ADEEB9E12E
:100D200080937F0590938005A0938105B093820501
:100D300085E0809388058DEE9EEFADEABEED809351
:100D4000830590938405A0938505B0938605E9E813
:100D5000F5E080E090E0863028F4DC01AE54BC4F32
:100D60002C9101C020E0219301968831910599F7DB
:100D700082E08093A1058AE08093A205089580EC2B
:100D800091EDA8E9BBE18093BF059093C005A093C6
:100D9000C105B093C20580E090E0A0E0B0E580938B
:100DA000C3059093C405A093C505B093C605E7ECB1
:100DB000F5E080E081938F5F8031E1F70895A0E056
:100DC000B0E0E5EEF6E00C941E2FD82F0E948329A8
:100DD0006115710581059105C9F30E94C12F10921B
:100DE0008305109284051092850510928605C4E053
:100DF000812C912C54018A94C0908305D090840555
:100E0000E0908505F0908605FE2CED2CDC2CCC24A2
:100E10000E94BC2FA50194010E94FD2E6C0D7D1D2A
:100E20008E1D9F1D609383057093840580938505B7
:100E300090938605C15001F7DD2309F450C009E8FD
:100E400015E0E801A12CB12C62E3C62ED12CE12CD7
:100E5000F12C8881882309F442C0B39419F40E94CC
:100E60007A063DC00E94BC2FA70196010E94FD2E6C
:100E7000E1E0E60FA9E8B5E08A2F801B8A1520F48F
:100E80008D918E13F9CFE9CF2091880530E0A0E154
:100E9000B7E20E94952E9B01AC01AE2FB0E00E94FC
:100EA000A42E40907F055090800560908105709041
:100EB0008205640D751D861D971D4090BF055090DD
:100EC000C0056090C1057090C205461657066806B9
:100ED000790618F2E993A39488E1A812BACFCDB7A6
:100EE000DEB7E0E10C943A2F8436910520F4BC0182
:100EF00080E090E017C09C018E3B910528F42A55B4
:100F00003109AAE0B0E00CC0823D910528F4245BD1
:100F10003109A4E6B0E004C02D5C3109A8E5B2E0D7
:100F20000E94952EA4E6B0E09B01AC010E94A42E85
:100F3000089590E08C599F4F0E947407089582E0B5
:100F40008093B00085E08093B10061E083E00E946F
:100F5000302A60E083E00E94692A08950097C9F072
:100F60009C0140E050E068E478EE81E090E00E946F
:100F7000FD2E2F3F31054105510529F020F02FEFBF
:100F800030E040E050E02093B3008091B0008061F9
:100F900003C08091B0008F7E8093B000089560E020
:100FA0008CE00E94302A61E08BE00E94302A61E0F0
:100FB0008DE00E94302A60E082E00E94302A61E0E9
:100FC00084E00E94302A089542E050E068E476E030
:100FD00080E00E94B3280895E3E0F0E089E0809388
:100FE0005700E491E67081E0E63009F080E0089572
:100FF000CF93DF93C82F0E94EC07882381F0DFB7DF
:1010000081E080937605F8940E94570688E18093EA
:101010006000C0936000C1110E945706DFBFDF91DE
:10102000CF9108958F929F92AF92BF92CF92DF920D
:10103000EF92FF92CF93FC01C0A5EC2FE770F0E098
:10104000E658FC4FA081B0E0C7FF03C024E130E0C8
:1010500002C02FE030E0FC0197A183E1989FF001EE
:101060001124E25CFE4F80809180A280B380A20FA9
:10107000B31F20E43FE14DE750E00E94AF2EA501F1
:1010800094010E94DB2E8C2F887149F469017A014A
:10109000E0EDCE0EE7E0DE1EE11CF11C1BC0C7FF39
:1010A00005C060E47AE88CE29EE004C060E07EEE79
:1010B0008AEB9BE069017A01F8EBCF0EFBE0DF1EC3
:1010C000E11CF11CA50194010E94DB2EC20ED31E6F
:1010D000E41EF51EC701B60169517C4F8F4F9F4F2B
:1010E00028EE33E040E050E00E94DB2EA8EEB3E0B3
:1010F0000E94A42ECF91FF90EF90DF90CF90BF90F1
:10110000AF909F908F9008958F3F910551F048F0D8
:10111000811522E0920738F08115934030F482E087
:10112000089580E0089581E0089583E00895A0E0A7
:10113000B0E0EDE9F8E00C94272FEB018A01B82F1D
:10114000B695A0E028813981F80120832A813B816E
:1011500021832C813D8122832E813F8123836881DD
:1011600079814A815B812C813D81EE81FF819F2FB6
:101170009295990F990F907C272F2370922B252FF2
:101180002370220F220F922B232F23702295207F72
:10119000922BF80194830B5F1F4F2896AF5FBA170D
:1011A00088F680FF24C0888199810E948408D82E07
:1011B0008A819B810E948408E82E8C819D810E94F7
:1011C0008408F82E8E819F810E948408F0E4DF9EBF
:1011D000A001112490E1E99E90011124242B282BD9
:1011E000E4E0FE9EB0011124262BF8012083CDB748
:1011F000DEB7E7E00C94432F803223E0920708F13A
:10120000883E23E0920740F48F519340E4E09695A6
:101210008795EA95E1F70895803D27E0920718F455
:101220008C5D93400895883928E0920768F4885CC3
:10123000974074E0969587957A95E1F78D509C4F8D
:10124000089580E090E008958FEF93E008958C304A
:10125000910540F4A4E0880F991FAA95E1F7885DF5
:101260009C4F0895843F23E0920718F484529C4FCA
:101270000895811524E0920740F48657934FF4E0D7
:10128000880F991FFA95E1F7089580E998E008958D
:101290009C013695279525753575821B930B9C010E
:1012A0002373337396958795969587958373937378
:1012B000820F931F9C0154E0369527955A95E1F7CC
:1012C000280F391F2F703F7041E051E0249FC0016B
:1012D000259F900D349F900D1124892F08952D98EE
:1012E000882319F000002B9A02C000002B98000000
:1012F0002D9A000008952D9A000083B12D980000CA
:10130000829581700895CF93DF93D82F5C9A2D98A2
:101310005C98C8E08D2F80780E946F09DD0FC15066
:10132000C9F72D98DF91CF9108958F770E94830997
:101330000895CF93DF93D82FC8E08D2F80780E9437
:101340006F09DD0FC150C9F72D98DF91CF91089536
:10135000CF93DF932D98C8E080E0D82FDD0F0E9457
:101360007B098D0FC150C9F7DF91CF9108950E947D
:1013700095090E94A8095C9A0895A1E0B0E0E3EC09
:10138000F9E00C942C2F806869830E94830969819D
:10139000862F0E9499095C9A2196E2E00C94482FCE
:1013A000CF93C0918305C827E82FF0E0E658FA4FA5
:1013B000678589E70E94BD096C2F8DE30E94BD09F6
:1013C0006C2F82E40E94BD09CF91089586E20E94AD
:1013D000B7090895CF93DF93EC016C818CE10E94F3
:1013E000BD096D818DE10E94BD096E818EE10E9473
:1013F000BD096F8180E20E94BD09688581E20E947B
:10140000BD09698582E20E94BD096A8583E20E9466
:10141000BD096B8584E20E94BD096C8585E20E944E
:10142000BD096D858AE20E94BD096E858EE60E9427
:10143000BD096F858FE60E94BD09688980E70E941B
:10144000BD09698981E70E94BD096A8982E70E9416
:10145000BD09DF91CF910895CF92DF92EF92FF9275
:10146000CF93DF936B017C01C11488E3D8068CE92C
:10147000E8068CE1F80628F5C701B60120E836E950
:1014800048E950E00E94DB2EE901689760E879E6C0
:1014900087E69FEF0E94B72E6C0D7D1D8E1D9F1D50
:1014A000F2E0660F771F881F991FFA95D1F721E7A1
:1014B00032E040E050E00E94DB2EF22EE32E80E48A
:1014C00021C0C701B60120E03DE241E351E00E94A6
:1014D000DB2EE901689760E073ED8EEC9EEF0E94D1
:1014E000B72E6C0D7D1D8E1D9F1D660F771F881FEB
:1014F000991F21E732E040E050E00E94DB2EF22EFF
:10150000E32E80E66C2F6F71680F85E70E94BD099E
:101510006E2D86E70E94BD096F2D87E70E94BD09E9
:10152000DF91CF91FF90EF90DF90CF900895682FDB
:101530008DE60E94BD0908958F929F92AF92BF924F
:10154000CF92DF92EF92FF92CF93DF93D82F61E09B
:1015500089E00E94692A62E370E080E090E00E94E6
:10156000A62960E089E00E94692A62E370E080E0D9
:1015700090E00E94A62983E00E94B7098093750538
:1015800084E00E94B7098093740560E086E00E94C1
:10159000BD0961E087E00E94BD096FE789E00E9414
:1015A000BD0965E08AE00E94BD0965E18BE00E940B
:1015B000BD0962E18CE00E94BD096DEF8DE00E94E3
:1015C000BD0960E08EE00E94BD09DD2319F08BE2C9
:1015D00091E008C02091A10533E1239FC0011124AF
:1015E000825C9E4F0E94EA096CE880E30E94BD097C
:1015F0006FE082E30E94BD0962E483E30E94BD09BB
:101600008091A20587FF02C064E101C06AE084E323
:101610000E94BD096AE285E30E94BD096DE286E38E
:101620000E94BD0964ED87E30E94BD0960E088E384
:101630000E94BD0960E089E30E94BD09D11109C083
:10164000C0908305D0908405E0908505F0908605D4
:1016500007C0C5E9CC2EC1ECDC2EED2CCEEDFC2E66
:10166000CAE38F2C9924AA24BB24682D8C2F0E94B6
:10167000BD09682D85E08C0F0E94BD09FE2CED2C64
:10168000DC2CCC24CF5FCE3361F76FEF83E40E9474
:10169000BD096FEF84E40E94BD096FEF85E40E94ED
:1016A000BD096FEF86E40E94BD09DD2311F066E0FD
:1016B00002C0609187058DE60E94BD0960E089E760
:1016C0000E94BD09609188058AE70E94BD0960E01B
:1016D00083E70E94BD0960E084E70E94BD09D11143
:1016E00009C060917F05709180058091810590917E
:1016F000820504C060EC72E98DEE99E10E942C0A2B
:10170000DF91CF91FF90EF90DF90CF90BF90AF909F
:101710009F908F90089561E087E00E94BD0964E288
:101720008EE70E94BD0963E088E00E94BD0960E089
:1017300088E00E94BD0965E087E00E94BD0962E083
:1017400085E00E94BD0983E00E94B709809375057A
:1017500084E00E94B70980937405089583E00E9495
:10176000B7098093750584E00E94B70980937405DA
:1017700061E087E00E94BD096AE070E080E090E0EF
:101780000E94A6290E948B0B00000895CF92DF9241
:10179000FF920F931F93CF93DF931F92CDB7DEB7C6
:1017A000082F162F8EE399830E94BD09F02EC02EBC
:1017B0009981D92E8C2D8F19811738F4F6016191FA
:1017C0006F018FE70E94BD09F5CF64E085E00E94BC
:1017D000BD0983E00E94B7098093750584E00E94EB
:1017E000B709809374050E948329609370057093F4
:1017F0007105809372059093730569E087E00E94FC
:10180000BD0981E0809377050F90DF91CF911F9103
:101810000F91FF90DF90CF9008950F931F930E9438
:10182000C60B80917705813099F40E94832900913D
:101830007005109171052091720530917305601B40
:10184000710B820B930B603A76488140910548F307
:1018500080917705813031F46EE971E086EE95E094
:101860000E946F2B1F910F9108950F931F938091EA
:101870007705823021F41092770581E020C08091B5
:1018800077058130D9F40E94832900917005109169
:1018900071052091720530917305601B710B820BED
:1018A000930B613A76488140910540F061E087E012
:1018B0000E94BD091092770582E001C080E01F916F
:1018C0000F910895CF93DF93EC014AE050E06D2F24
:1018D00070E086EE95E00E943D2C6EE286EE95E08B
:1018E0000E94412BBE0184E0769567958A95E1F7C9
:1018F0006F7077274AE050E086EE95E00E943D2C1D
:101900006EE286EE95E00E94412BBE016F70772754
:101910004AE050E086EE95E00E943D2CDF91CF91A9
:101920000895D82FC0E0CD1780F45E9A64E670E089
:1019300080E090E00E94A6295E9864E670E080E076
:1019400090E00E94A629CF5FEECF6CE271E080E0CC
:1019500090E00E94A629E6CF0F931F93CF93DF93C9
:10196000EC01062F15E0115051F0CE010E943831E4
:10197000081741F0602FCE010E944031F4CF82E081
:101980000E94910CDF91CF911F910F910895A0E0DB
:10199000B0E0EDECFCE00C941E2F482E562EC0E07B
:1019A000D0E0612C712CE12CF12C00E010E0411012
:1019B0000CC06090D80586E4689E3001112459E17E
:1019C000E52EF12C0EEB15E01EC091E049120FC080
:1019D0006090D805E6E46E9E30011124FBE16F0EA5
:1019E000711C49E2E42EF12C0AE715E00CC082E0FC
:1019F000481209C028E1622E77247394EE24E39400
:101A0000F12C07ED15E043018C0E9D1E1092790517
:101A1000109278053401A62CA818B12CC3010196A8
:101A20006C01AE14BF04A8F4A00EB11E511006C084
:101A3000C3010E943831F501808305C0F501608142
:101A4000C3010E94AC0CF50180810E946106360141
:101A5000E2CFC301511018C0C3010E943831B82E23
:101A6000C6010E9438312B2D30E0322F2227282B3F
:101A700080917805909179058217930779F4C0E0F9
:101A8000D0E05524539493CF3601609179050E949C
:101A9000AC0C60917805C6010E94AC0CC05EDE4FB4
:101AA000C13E92E0D90708F482CF852DCDB7DEB7CD
:101AB000E0E10C943A2F61E082E00E94C70C0895A7
:101AC00060E082E00E94C70C8091D705853020F04D
:101AD0001092D7050E945B0D8091D7058093D805A1
:101AE000089561E080E00E94C70C61E081E00E94FF
:101AF000C70C089560E080E00E94C70C882351F075
:101B000060E081E00E94C70C882321F080917A0573
:101B1000883349F00E94BF060E947A0681E00E9445
:101B2000DF060E94710D0895882319F06AEA71E0BA
:101B300002C06EEA71E086EE95E00E946F2B089578
:101B4000FF920F931F93CF93DF9369EC7BE086EEB8
:101B500095E00E941B2B40917F055091800560917C
:101B60008105709182052AE030E086EE95E00E94C2
:101B7000442C63EB7BE086EE95E00E941B2B4091AA
:101B8000830550918405609185057091860520E15B
:101B900030E086EE95E00E94442C6DE97BE086EE15
:101BA00095E00E941B2B4AE050E06091870586EE8D
:101BB00095E00E946C2C67E87BE086EE95E00E9441
:101BC0001B2B4AE050E06091880586EE95E00E946C
:101BD0006C2C61E77BE086EE95E00E941B2BC9E848
:101BE000D5E0F12C8E0188818823A9F0FF2031F007
:101BF00061EB71E086EE95E00E943E2B21964AE073
:101C000050E0F801608186EE95E00E94352CF39457
:101C1000F8E1FF12E7CF86EE95E00E94492B6BE5D5
:101C20007BE086EE95E00E941B2B4AE050E060913D
:101C3000A10586EE95E00E946C2C66E47BE086EEC2
:101C400095E00E941B2BE091A205E770F0E0EE0FFB
:101C5000FF1FEE57FC4F6081718186EE95E00E9478
:101C60006F2B61E37BE086EE95E00E941B2B809159
:101C7000A2058871883069F028F4811113C068E2E8
:101C80007BE00CC0803141F0883161F46CE07BE096
:101C900005C06CE17BE002C066E17BE086EE95E08A
:101CA0000E945D2B68EF7AE086EE95E00E941B2B88
:101CB00040917B0550917C0560917D0570917E057A
:101CC0002AE030E086EE95E00E94442C6FED7AE049
:101CD00086EE95E00E941B2B8091C30580710E94C7
:101CE000940D66EC7AE086EE95E00E941B2B8091C5
:101CF000C30580740E94940D6DEA7AE086EE95E04B
:101D00000E941B2B8091C30580720E94940D60E994
:101D10007AE086EE95E00E941B2B8AE795E00E9410
:101D20001208AB01BC012AE030E086EE95E00E948B
:101D3000262C6BE87AE086EE95E00E941B2B8AE762
:101D400095E00E9412089B01AC0160E472E48FE010
:101D500090E00E94DB2EBA01A9012AE030E086EE75
:101D600095E00E94262C68E87AE086EE95E00E94D5
:101D70005D2BCDB7DEB7E5E00C94452F8F929F9297
:101D8000AF92BF92CF92DF92EF92FF92811107C084
:101D90006FE77AE086EE95E00E945D2B2FC090E021
:101DA0000E94740724E630E040E050E00E94DB2E01
:101DB000CA01B9012AE030E040E050E00E94DB2E89
:101DC00049015A016B017C012AE030E0B501A40110
:101DD00086EE95E00E94262C6EE286EE95E00E944B
:101DE000412B2AE030E0B701A60186EE95E00E9483
:101DF000262C63E786EE95E00E94812BFF90EF9002
:101E0000DF90CF90BF90AF909F908F9008951F93D9
:101E1000CF93DF9365E77AE086EE95E00E941B2B77
:101E20008091A305813041F46CE57AE086EE95E07F
:101E30000E945D2B10E050C0823019F465E47AE016
:101E4000F5CF843019F461E37AE0F0CF853091F773
:101E500066E27AE0EBCFC12FD0E0C930D1050CF4B7
:101E600041C068E3610F86EE95E00E94412B6EE170
:101E70007AE086EE95E00E941B2BBE016F5F7F4FDC
:101E80004AE050E086EE95E00E94052C63E17AE09E
:101E900086EE95E00E941B2BCD55DA4FE981E032AA
:101EA00018F566E07AE086EE95E00E941B2B8981AA
:101EB000803130F06DE673E086EE95E00E943E2BB7
:101EC00069816F7070E06F5F7F4F4AE050E086EE8F
:101ED00095E00E940E2C1F5F80914C05181708F4A6
:101EE000BACF0FC061E3BECFEF70F0E0EE0FFF1F7F
:101EF000EE56FC4F6081718186EE95E00E946F2B5B
:101F0000EACF6BEE79E086EE95E00E941B2B809184
:101F1000BB050E94BE0E60ED79E086EE95E00E9462
:101F20001B2B8091BC050E94BE0E65EB79E086EE0E
:101F300095E00E941B2B8091BD050E94BE0E6AE9B0
:101F400079E086EE95E00E941B2B4091B3055091FD
:101F5000B4056091B5057091B6054115510561054F
:101F6000710539F12AE030E086EE95E00E94442CBC
:101F700067E679E086EE95E00E941B2B8091B7051D
:101F80000E949907AB01BC012AE030E086EE95E0A3
:101F90000E94442C63E479E086EE95E00E941B2BBE
:101FA0004AE050E06091B80586EE95E00E946C2C06
:101FB00006C06AE379E086EE95E00E945D2B6DE154
:101FC00079E086EE95E00E941B2B6091B905709137
:101FD000BA054AE050E086EE95E00E94562C60E09B
:101FE00079E086EE95E00E941B2B6091B20560348B
:101FF00050F470E06F5F7F4F4AE050E086EE95E06E
:102000000E940E2C06C067EF78E086EE95E00E94F5
:102010005D2B6AED78E086EE95E00E941B2B8091A7
:10202000B10580FF03C063EB71E002C067EB71E0B4
:1020300086EE95E00E946F2B6DEB78E086EE95E0E2
:102040000E941B2B8091B10582700E94940D6EE955
:1020500078E086EE95E00E941B2B8091B10584709C
:102060000E94940D6FE778E086EE95E00E941B2BAE
:102070008091B10588700E94940DDF91CF911F91DE
:1020800008950F931F93CF93DF93209149052F3F1E
:10209000A9F56FEF75E086EE95E00E941B2B88E8AE
:1020A00093E00E94620C6EED75E086EE95E00E9472
:1020B0001B2B80914A0590914B050E94620C6BEAA4
:1020C00075E086EE95E00E945D2B68E875E086EE8F
:1020D00095E00E945D2B60E775E086EE95E00E943A
:1020E0005D2B6BE475E086EE95E00E945D2B86EE3D
:1020F00095E00E94492B0E94070F68C012160CF051
:1021000065C0332727FD309580914C0590E08217FC
:1021100093070CF45BC066E375E086EE95E00E94E1
:102120001B2B60914905772767FD70954AE050E0C9
:1021300086EE95E00E940E2C6BE075E086EE95E051
:102140000E941B2B10E008E280914D051817D0F576
:10215000C12FD0E0CC0FDD1FC25BDA4F288130E009
:1021600080914905992787FD909501972817390790
:1021700039F56BEB71E086EE95E00E943E2B4AE06C
:1021800050E0602F86EE95E00E94352C6FEB71E0F9
:1021900086EE95E00E943E2BE981EF70F0E0EE0FB5
:1021A000FF1FEE56FC4F6081718186EE95E00E9424
:1021B0003E2B63EC71E086EE95E00E943E2B0F5FB4
:1021C0001F5FC2CF86EE95E00E94492BDF91CF9131
:1021D0001F910F910895FF920F931F93CF93DF9359
:1021E000C9E8D5E0F12C8E0188818823D1F165EC16
:1021F00071E086EE95E00E943E2B4AE050E06F2DA4
:1022000086EE95E00E94352C62ED71E086EE95E059
:102210000E943E2B2196F801208130E0A0E1B7E238
:102220000E94952E9B01AC01A0918805B0E00E9410
:10223000A42EAB01BC0180917F0590918005A091F7
:102240008105B0918205480F591F6A1F7B1F2AE044
:1022500030E086EE95E00E94442CF394F8E1FF1202
:10226000C2CFCDB7DEB7E5E00C94452F1092E30462
:1022700085E6E4EEF4E0DF011D928A95E9F7089522
:10228000CF93C82F8F3719F0883009F045C0E091FF
:10229000E304EE23D9F1E150E093E304F0E0EC51E4
:1022A000FB4F10826DE070E086EE95E00E945906CB
:1022B000C0E08091E304C81760F4EC2FF0E0EC512B
:1022C000FB4F608170E086EE95E00E945906CF5F7B
:1022D000F0CF60E270E086EE95E00E9459066DE076
:1022E00070E086EE95E00E945906C0E08091E3041C
:1022F000C81778F5EC2FF0E0EC51FB4F608170E0EF
:1023000086EE95E00E945906CF5FF0CF67E086EE3B
:1023100095E00E94412B1DC08B3119F40E943611AB
:102320001AC08D30C1F08A30B1F08091E304843658
:1023300068F76C2F70E086EE95E00E945906E091F8
:10234000E30481E08E0F8093E304F0E0EC51FB4F57
:10235000C08380E001C081E0CF910895CF93C82F62
:102360000E9483296093CC047093CD048093CE04A3
:102370009093CF04C093E104CC2329F040E051EEC8
:1023800060E070E004C040E855E260E070E086EE96
:1023900095E00E94CB2DCF9108959091D004492FC4
:1023A0004F7050E0BA016F5F7F4F292F30E0E4E0BB
:1023B00035952795EA95E1F76217730759F0FA0109
:1023C000EF52FB4F808381E0890F8F70907F892BC4
:1023D0008093D00408956EE770E086EE95E00E9449
:1023E00059060895A3E1B1E0E8EFF1E10C941F2F45
:1023F000E9E8F5E0712C8191882321F0739428E1BC
:102400007212F9CF66ED71E086EE95E00E946F2BB7
:102410004AE050E0672D86EE95E00E946C2C80E04B
:102420000E949C0A0E948B0B8E010E5F1F4FC12CD5
:10243000D12C7601C39466246A945C2C0E9477297F
:102440004B015C012091880530E0A0E1B7E20E94D9
:10245000952E9B01AC01C701B6010E94B72E2091B9
:102460007F05309180054091810550918205620F72
:10247000731F841F951F2091BF053091C0054091A7
:10248000C1055091C205261737074807590718F4A8
:10249000F801608225C08C2D0E94D00961E070E0B7
:1024A00080E090E00E94A629F80110820E9477291E
:1024B000681979098A099B09643F71408105910572
:1024C00040F40E94E609F8019081981778F780831C
:1024D000EDCF50FE03C05D985E9A02C05D9A5E9893
:1024E0002FEFC21AD20AE20AF20A0F5F1F4F8FEFD4
:1024F000C816D104E104F10409F09FCFCE019395F1
:10250000FC01D82E7FEF68EC2E2F281B271510F02A
:1025100051E056C0DE01129651E02FEF41E03D91AF
:10252000321710F0322F01C0452F5F5F5F3F11F06F
:10253000232FF5CF4193242F30E0A1E0B0E0AC0F82
:10254000BD1FA20FB31F5C93413079F0DE01A20FD3
:10255000B31F5C93423049F0AFEFBFEFAC0FBD1F2C
:10256000A20FB31F6C934E3F78F6A2E0B0E0AC0F21
:10257000BD1FA20FB31F7C934D3F30F6A3E0B0E028
:10258000AC0FBD1FA20FB31F6C93BECF452F242FDE
:1025900030E0FC01E20FF31F6081AFEFB0E0AC0F61
:1025A000BD1FA20FB31F2C91621748F44150DC01EC
:1025B000A40FB11D2C9120836C934111E8CF5F5F74
:1025C000571520F3372D369520E0231770F4DC01E2
:1025D000A20FB11D4C91522F530FFC01E50FF11DBD
:1025E00050815C9340832E5FF0CFF9E8EF2EF5E049
:1025F000FF2E8C01802F8D19871598F4F801C1905A
:102600008F014AE050E06C2D86EE95E00E94352C5B
:102610006CE286EE95E00E94412BF701C1927F01AA
:10262000E9CF86EE95E00E94492B81E0CD5EDE4F3A
:10263000EFE00C943B2F1F920F920FB60F921124D4
:102640001F932F933F934F935F936F937F938F933A
:102650009F93AF93BF93CF93DF93EF93FF93C0917B
:102660008600D09187008091870490918804209102
:10267000A904211155C09E01281B390B8091C30567
:102680009091C405A091C505B091C60585FD02C015
:1026900036952795253C49E03407B8F140910A0169
:1026A00050E060E070E02CE1B695A795979587958E
:1026B0002A95D1F70097A105B10521F481E090E0BA
:1026C000A0E0B0E084179507A607B707D8F480917B
:1026D0000A018F3FB9F040E080910A01481780F469
:1026E000842F90E0880F991FFC01E757FB4F208152
:1026F0003181FC01E55FFE4F318320834F5FECCFDA
:102700001092AA0410920A010BC02D3B82E03807F8
:1027100020F080910A018031D8F08FEF80930A0178
:10272000D0938804C0938704FF91EF91DF91CF91FC
:10273000BF91AF919F918F917F916F915F914F91D9
:102740003F912F911F910F900FBE0F901F901895E2
:1027500010910A0181E0810F80930A01C9010E9452
:10276000FC08E12FF0E0EE0FFF1FE757FB4F9183CE
:102770008083D6CF83E0809380008AE980938100B4
:102780008091C30586FD05C080918100806480939F
:1027900081008FEF9FEF9093890080938800809154
:1027A0006F00806280936F000895CF93DF930E9443
:1027B000600D8091D805843039F58FE00E949C2A05
:1027C000C1E0D0E0892B11F4C0E0D0E080E10E94AC
:1027D0009C2A892B19F082E090E002C080E090E012
:1027E0008C2B9D2B8230910539F08330910539F087
:1027F000019739F481E006C01092D80505C082E047
:1028000001C083E08093D805DF91CF9108956F30A8
:1028100018F086958058089589E0689F802D1124CE
:102820000895A0E0B0E0E7E1F4E10C94262FC82F72
:102830000E948329009138041091390420913A04B0
:1028400030913B046B017C01C01AD10AE20AF30A01
:102850009701860149E8C41643E1D406E104F10476
:1028600010F010923C046093380470933904809304
:102870003A0490933B042091A9048FEF820F823099
:10288000E8F5E0913C04EE2309F46EC1E13011F467
:1028900082E0D8C1E03178F581E08E0F80933C046E
:1028A000F0E0E757FB4FC083803109F0D4C1EBE87B
:1028B000F4E0213029F4A181A695A695808108C075
:1028C00080819181A92FA695A695A6959695879525
:1028D000A03148F4B0E090E0AA0FBB1FA55FBE4F47
:1028E00011969C938E931092AA04329684E0E93953
:1028F000F807F9F6B0C110923C04ADC1233009F0DD
:1029000023C1E0913C04E11118C0CF3009F011C19E
:102910000E9477290091B7041091B8042091B9045E
:102920003091BA04601B710B820B930B62307105FE
:102930008105910508F089C1FCC0E73148F481E0C8
:102940008E0F80933C04F0E0E857FB4FC083F1C04A
:10295000E73109F0ECC0C111EAC040E050E0ABE063
:10296000CA01B3E0880F991FBA95E1F7A49F9001BF
:10297000A59F300D1124F901E757FB4F6081E181DC
:102980007E2F777075956795FC01EE0FFF1FE55F51
:10299000FE4F71836083F901E657FB4FB081B69516
:1029A000B695B695E181FE2FF295FF0FF07E6F2F61
:1029B0006B2BE695E695E6957E2F77707595679576
:1029C000FC01EE0FFF1FE35FFE4F71836083F9018F
:1029D000E557FB4FB081B295B695B695B370C181FE
:1029E000DC2FDD0FDD0F6D2F6B2BC295C695C695C5
:1029F000C370E281E170EE0FEE0F7E2F7C2B759598
:102A00006795FC01EE0FFF1FE15FFE4F718360834E
:102A1000F901E357FB4FB081B695E181FE2FF795A1
:102A2000FF27F7956F2F6B2BE6957E2F77707595A7
:102A30006795FC01EE0FFF1FEF5EFE4F7183608311
:102A4000F901E257FB4FB081B295BF70E181FE2FD3
:102A5000F295F07F6F2F6B2BE295EF707E2F7770E2
:102A600075956795FC01EE0FFF1FED5EFE4F7183BC
:102A70006083F901E157FB4FB081BB1FBB27BB1F30
:102A8000C181DC2FDD0F6D2F6B2BCC1FCC27CC1F12
:102A9000E281E370EE0F7E2F7C2B75956795FC012C
:102AA000EE0FFF1FEB5EFE4F71836083F901EF565F
:102AB000FB4FB081B695B695E181FE2FF295FF0FE1
:102AC000FF0FF07C6F2F6B2BE695E6957E2F7770CE
:102AD00075956795FC01EE0FFF1FE95EFE4F718350
:102AE0006083F901EE56FB4F2081229526952770D1
:102AF0003181E32FEE0FEE0FEE0F6E2F622B732F4F
:102B000072957695777075956795FC01EE0FFF1FAE
:102B1000E75EFE4F718360834F5F5F4F4230510528
:102B200009F01ECF80919F0483FF1092AA04109297
:102B30003C040E9477296093B7047093B804809393
:102B4000B9049093BA0487C0243009F084C060911E
:102B50003C0461110BC0C83AB1F41092790510928F
:102B6000780588EA0E94610681E06CC0613019F442
:102B7000C093370404C0623031F4C09336048C2F04
:102B80000E9461065AC0E09136042E2F30E0220FD9
:102B9000331F462F50E0C9010296841795073CF079
:102BA000633268F7FA01EA57FB4FC083E8CF2D5F25
:102BB0003F4F8C2F90E06091780570917905421716
:102BC000530749F4982F88278627972790937905EC
:102BD0008093780532C06817790769F580913704CA
:102BE000813049F5E13118F080E180933604F090AE
:102BF0003604CAE8D4E000E010E00F15D0F4FE017E
:102C00003197808190E0982F88272881822B63E07C
:102C1000969587956A95E1F70E94FC08F801EE0FFA
:102C2000FF1FE55FFE4F918380830F5F1F4F22964A
:102C3000E4CF1092AA0410923C0480913C048823B3
:102C400051F08F5F80933C0406C080913C048F5FFD
:102C500080933C046ECFCDB7DEB7E8E00C94422FF2
:102C6000CF93DF93E82FF0E0E254FA4FE185E031B3
:102C700050F4F894F0E0EE0FFF1FE55FFE4F808107
:102C8000918178945DC08EE08E0F8B3058F4F0E027
:102C9000E25FF10924E62E9FC0012F9F900D1124C1
:102CA0000C964EC0E03F09F446C038F4E13181F0A3
:102CB000E23191F0E03139F409C0ED3FB1F1EE3F7E
:102CC000B9F1E13F79F180E092E03AC082E101C0E0
:102CD00083E10E94C52A34C08FE00E949C2AC1E093
:102CE000D0E0892B11F4C0E0D0E080E10E949C2A62
:102CF000892B19F082E090E002C080E090E08C2BFC
:102D00009D2B8230910541F08330910541F0019770
:102D1000A9F086EA92E014C08CE090E011C089E549
:102D200091E00EC086E090E00BC08AEF93E008C00F
:102D30008FEF93E005C080E090E002C084EF93E065
:102D4000DF91CF910895A2E2B0E0E9EAF6E10C94B8
:102D50001C2F9E012F5F3F4F80E1D9011D928A9564
:102D6000E9F764E072E086EE95E029A33AA30E94B9
:102D70006F2B0E94AE0B1D8A1E8A1F8A188E312C63
:102D8000212C00E0812C912C540170E4472E71EE2F
:102D9000572E7DE9672E78E1772EE0E5CE2EE3EC25
:102DA000DE2EE12CF12C84EF91E0A0E0B0E08D8FDD
:102DB0009E8FAF8FB8A380EC91EDA8E9BBE1898F1E
:102DC0009A8FAB8FBC8F80E491EEADE9B8E1898B2F
:102DD0009A8BAB8BBC8B86EE95E00E94832C892B63
:102DE00009F4E1C086EE95E00E94B02C9C013327E7
:102DF0002C32310509F442C0ACF42332310509F01C
:102E0000ABC019821A821B821C821D821E821F8205
:102E1000188619861A861B861C861D861E861F86A6
:102E2000188A60C02434310529F02335310509F4AE
:102E3000B2C092C064E486EE95E00E94412B2AE085
:102E400030E040E451EE6DE978E186EE95E00E94D5
:102E5000CF2B6CE286EE95E00E94412B2AE030E019
:102E600040EC51ED68E97BE186EE95E00E94CF2BC6
:102E70006CE286EE95E00E94812BADCF0F5F0430AF
:102E800009F0A9CF29813A814B815C81A8EEB3E09A
:102E90000E94A42E698B7A8B8B8B9C8B2D813E811B
:102EA0004F8158850E94A42E698F7A8F8B8F9C8FBB
:102EB00029853A854B855C852D8F3E8F4F8F58A392
:102EC0002D853E854F8558890E94A42E6B017C017B
:102ED00060323EE473078105910530F462E38CE1D2
:102EE0000E94BD0900E077CF603345E77407810594
:102EF000910510F462E2F3CF60345CE97507810557
:102F0000910510F466E2EBCF80E5C81683ECD80695
:102F1000E104F10410F462E1E2CF90E6C9169AEE02
:102F2000D906E104F10410F465E1D9CFA0E7CA168F
:102F3000A1E1DA06A1E0EA06F10410F461E0CFCFE6
:102F4000B0EACB16B6E8DB06B1E0EB06F10410F40C
:102F500063E0C5CF65E0C3CF10ED180F1A3008F05D
:102F60003ACFE1E0F0E0EC0FFD1F24E0029FE00D1E
:102F7000F11D11242081318142815381AAE0B0E00A
:102F80000E94A42E610F711D811D911D60837183AC
:102F90008283938320CF49885A886B887C88812CD0
:102FA000912C540118CF81149104A104B10489F427
:102FB000C301B2010E942C0A61E070E080E090E061
:102FC0000E94A6291D8A1E8A1F8A188E312C22244F
:102FD0002A948D8D9E8DAF8DB8A188169906AA066C
:102FE000BB06D0F40E94E6092D893E894F89588D91
:102FF000280F311D411D511D2D8B3E8B4F8B588F3E
:10300000381608F4382E821508F4282E3FEF831A5C
:10301000930AA30AB30A56C0C301B20128EE33E0F3
:1030200040E050E00E94DB2EBA01A9012AE030E026
:1030300086EE95E00E94262C6CE286EE95E00E94DA
:10304000412B4AE050E0632D86EE95E00E94352C3E
:103050006CE286EE95E00E94412B6D897E898F8916
:10306000988DA50194010E94DB2EBA01A9012AE0E6
:1030700030E086EE95E00E94262C6CE286EE95E02C
:103080000E94412B4AE050E0622D86EE95E00E94BE
:10309000352C6CE286EE95E00E94812B4C0C5D1C79
:1030A0006E1C7F1C898D9A8DAB8DBC8D841595050A
:1030B000A605B70520F449885A886B887C88812C3E
:1030C000912C540129893A894B895C89283E3340E7
:1030D0004105510509F07FCEA296E2E10C94382F0C
:1030E000ACE1B0E0E6E7F8E10C94262F0E948329DA
:1030F0006B017C0181E00E949C0A14E703E01983C4
:1031000061E0CE0101960E940D0C009377050E94AC
:103110008B0B6AEF70E080E090E00E94A62980911E
:103120007705833089F486EE95E00E94832C892B05
:1031300059F40E9483296C197D098E099F09603812
:10314000734C894C9140D8F280917705833009F413
:103150004FC08FE70E9495090E94A8098983843592
:1031600011F083E05CC00E94A80910924A05809388
:103170004B050E94A80920914A0530914B05280F64
:10318000311D30934B0520934A050E94A809809376
:103190004C050E94A80980934D05813110F7F12C50
:1031A0000F2D10E080914D0590E0880F991F0817B2
:1031B000190740F40E94A809F801E25BFA4F8083E6
:1031C000F394EECF80E7898361E0CE0101960E94FF
:1031D0000D0C83E0809377050E948B0B62E370E017
:1031E00080E090E00E94A62980917705833011F459
:1031F00082E015C08FE70E9495090E94A809898383
:10320000803509F0AECF03EA15E00E94A809F80165
:1032100081938F01F5E00E3B1F07B9F781E06C96B3
:10322000E8E00C94422F80914905992787FD9095FD
:10323000A92FB92FFC013196EB30F10508F066C0DB
:10324000EC5CFF4F0C94532F62E778E086EE95E03C
:103250000E945D2B88E893E00E94620C6AE578E0AA
:1032600086EE95E00E945D2B65E378E086EE95E0C2
:103270000E945D2B6BE078E086EE95E00E945D2B6E
:103280006AEE77E086EE95E00E945D2B6DEB77E0CD
:1032900086EE95E00E945D2B67E977E086EE95E08B
:1032A0000E945D2B63E777E086EE95E00E945D2B40
:1032B0006CE477E086EE95E00E945D2B86EE95E06B
:1032C0000E94492B0E94A00D21C06FE277E01AC036
:1032D0006AE077E017C065EF76E014C066ED76E04F
:1032E00011C062E976E00EC06DE776E00BC068E6DB
:1032F00076E086EE95E00E945D2B62E276E002C009
:103300006CE076E086EE95E00E945D2B6AE070E06E
:1033100080E090E00E94A62986EE95E00E94832C32
:10332000892B29F086EE95E00E94B02CF5CF089508
:10333000ACE1B0E0EEE9F9E10C94262F909149055B
:103340009F3F09F023C1482F50E0FA013A97EF362A
:10335000F10508F00FC1E15CFF4F0C94532F61E1C0
:1033600072E0A0C06DE172E086EE95E00E946F2BE6
:1033700085E789838BE1E3EAF5E0DE0112960190AF
:103380000D928A95E1F76CE1CE0101960E940D0C39
:103390000E948B0B83E08093770568EC70E080E0FF
:1033A00090E00E94A62980917705843009F0E2C060
:1033B0008FE70E9495090E94A8098983853509F045
:1033C000D9C06DEE74E086EE95E00E945D2B6FEC47
:1033D00074E086EE95E00E945D2B61EB74E096C090
:1033E00065E372E086EE95E00E946F2B89E68983A3
:1033F00061E0CE0101960E940D0C0E948B0B83E0D0
:103400008093770568EC70E080E090E00E94A62948
:1034100080917705843009F0ADC08FE70E9495094F
:103420000E94A80989838E010E5F1F4F7E014DE126
:10343000E40EF11C0E94A809F80181938F01EE159A
:10344000FF05C1F78BE1FE013296A3EAB5E00190DA
:103450000D928A95E1F78981893409F08BC063E97F
:1034600074E086EE95E00E945D2B65E774E086EEE1
:1034700095E00E945D2B67E574E048C06FE472E060
:1034800086EE95E00E946F2B8EEF8093490572C007
:1034900080528750805390914C05981708F066C071
:1034A0006EE572E086EE95E00E946F2B63C084E1CA
:1034B0008093490560E274E029C085E18093490565
:1034C00069EE73E023C086E18093490562EB73E007
:1034D0001DC087E18093490568E673E017C088E165
:1034E0008093490567E573E011C089E18093490540
:1034F00063E473E00BC08AE1809349056EE273E0F8
:1035000005C08BE18093490566E073E086EE95E0A7
:103510000E945D2B2FC06CEE72E086EE95E00E945B
:103520005D2B8091B10591E01DC066ED72E086EEE5
:1035300095E00E945D2B8091B10592E013C061EC93
:1035400072E086EE95E00E945D2B8091B10594E0DB
:1035500009C066EA72E086EE95E00E945D2B8091DC
:10356000B10598E089278093B1058FEF80934905D5
:103570000E94411086EE95E00E94832C892B09F46D
:103580005BC186EE95E00E94B02CF4CF0E94401102
:10359000882309F451C18091E304811104C08FEFA5
:1035A0008093490541C140E050E060E070E084EE66
:1035B00094E00E94CA2F40914905042F112707FD6E
:1035C0001095212F312FF8013197EB31F10508F0DB
:1035D0001BC1E255FF4F0C94532F552747FD5095C3
:1035E00020914C0530E0241735070CF40DC18B01F8
:1035F0009C010150110921093109003211052105F1
:10360000310558F0C0904D05EFE4F5E0F12CD12CD8
:10361000A8E2EA2E415051090FC0FA01ED55FA4FC8
:1036200061506083D9C0DF0111972C9130E02417DD
:10363000350729F0F3943296FC10F5CFCBC00E2D50
:1036400010E020E030E0061717072807390741F49B
:103650002081DA01AD55BA4F11962C93DD24D39415
:10366000E394E8CF6F3F71058105910511F008F0F3
:10367000CBC06093BB05B0C06F3F7105810591055C
:1036800011F008F0C1C06093BC05A6C06F3F710582
:103690008105910511F008F0B7C06093BD059CC08D
:1036A0002091E40420622037E9F440E050E060E03B
:1036B00070E085EE94E00E94CA2F9B01AC01DC0112
:1036C000CB010197A109B1090897A105B10508F03F
:1036D000AEC0A4EDB0E30E94A42E6A5E7C4A8A4686
:1036E000954E24C02636E9F440E050E060E070E0FA
:1036F00085EE94E00E94CA2F9B01AC01DC01CB0156
:103700000197A109B1090797A105B10508F08FC07C
:10371000A8EAB1E60E94A42E645E7C438E46944ED5
:1037200005C0611571058105910579F08B019C013A
:103730000054114E2D4938410138F0EF1F07FAEFC0
:103740002F07F2E03F0708F05FC06093B305709366
:10375000B4058093B5059093B6053EC06F3F7105E3
:103760008105910511F008F04FC06093B70534C092
:103770008B019C0101501109210931090F3F1105ED
:103780002105310508F040C06093B80525C08B01C4
:103790009C01045C1940210931090D344DE11407E5
:1037A0002105310528F47093BA056093B90514C05A
:1037B000611571058105910521F48FEF8093B205A4
:1037C0000BC06134710581059105F0F4615060937F
:1037D000B20502C0DD20C1F08091E20481111AC05F
:1037E0008091830590918405A0918505B09186050F
:1037F0000196A11DB11D8093830590938405A0932C
:103800008505B093860506C060E772E086EE95E018
:103810000E946F2B0E9436118FEF809349056AE05A
:1038200086EE95E00E94812B0E94411005C061E068
:1038300070E080E090E07ACF6C96E8E00C94422F44
:103840006AE572E086EE95E00E945D2B62E472E02C
:1038500086EE95E00E945D2B86EE95E00E94832C1B
:10386000892B31F086EE95E00E94B02C0E949819C9
:103870000E947018823029F0833051F46DE072E0BC
:1038800002C064E272E086EE95E00E945D2B08952E
:103890008FEF809349051092E2040E9441108091BD
:1038A00049058E3F69F086EE95E00E94832C892BB6
:1038B000B1F386EE95E00E94B02C0E949819EFCFEC
:1038C00008950F931F93109149051F3F09F0D2C02F
:1038D000893409F457C000F5883309F469C058F4F5
:1038E000803309F477C008F061C08B3109F440C01F
:1038F0008132B1F1B9C0813409F487C030F4893321
:1039000009F466C0803461F1AFC0823409F48EC01E
:10391000863409F448C0A8C0823609F487C078F418
:10392000883531F128F48235C1F18335E1F09CC04E
:103930008A3509F494C0813609F467C095C082378E
:1039400061F128F4863679F18936E1F08DC0883747
:1039500079F08A3709F483C0833709F085C003C042
:1039600061E172E015C00E94710D6EE872E004C062
:103970000E947A0D68EA72E086EE95E00E946F2B55
:103980008EEF70C00E947A060E94BF0667EC72E05C
:1039900086EE95E00E946F2B67C081E00E94DF06F3
:1039A00060EE72E0F5CF0E94EB105EC080535AC00B
:1039B0006AEF71E086EE95E00E945D2B9091A20582
:1039C00088E0890F8871977E892B8093A2051AC0A1
:1039D00089E048C067EE71E086EE95E00E945D2BBD
:1039E0008091C3059091C405A091C505B091C6050D
:1039F00020E182278093C3059093C405A093C50559
:103A0000B093C605109349052FC061ED71E086EEB5
:103A100095E00E945D2B8091C3059091C405A09113
:103A2000C505B091C60540E4842710C060EC71E084
:103A300086EE95E00E945D2B8091C3059091C405B0
:103A4000A091C505B091C60520E282278093C305E9
:103A50009093C405A093C505B093C60502C00E940B
:103A6000201C8FEF80934905809149058E3F09F016
:103A7000D4C0DDC00E944011882309F4D8C08091D1
:103A8000E304811104C08FEF80934905C6C040E074
:103A900050E060E070E084EE94E00E94CA2F009154
:103AA0004905112707FD1095212F312FF801319776
:103AB000E930F10508F0B4C0E753FF4F0C94532FE1
:103AC0008B019C010154114E2D4938410F37104F85
:103AD0002A4F324008F0A4C060937F0570938005A0
:103AE000809381059093820577C0609383057093DE
:103AF0008405809385059093860581E08093E20498
:103B00006BC0683071058105910508F089C060932C
:103B1000870562C08B019C010150110921093109FF
:103B20000A3011052105310508F07AC06093880537
:103B300053C061EB71E084EE94E00E94043110E028
:103B4000009799F00E94DE30009779F0183130F438
:103B5000E12FF0E0E658FA4F87871F5F61EB71E0D5
:103B600080E090E00E940431EBCF1831A8F5E12FFE
:103B7000F0E0E658FA4F17861F5FF7CF6530710502
:103B80008105910508F04CC06093A10525C08B010B
:103B90009C01015011092109310906301105210547
:103BA0003105F0F52091A205287F262B2093A20550
:103BB00013C08B019C010150110921093109011524
:103BC000124C2140310560F560937B0570937C05B4
:103BD00080937D0590937E058091E204811113C04E
:103BE0008091830590918405A0918505B09186050B
:103BF0000196A11DB11D8093830590938405A09328
:103C00008505B09386050E9436118FEF8093490594
:103C10006AE086EE95E00E94812B0E94131907C08E
:103C200060E772E086EE95E00E946F2BECCF1F916B
:103C30000F9108958FEF809349051092E2040E943E
:103C40001319809149058E3F69F086EE95E00E9438
:103C5000832C892BB1F386EE95E00E94B02C0E9454
:103C6000611CEFCF6AE070E080E090E00E94A6293E
:103C700086EE95E00E94832C892B29F086EE95E054
:103C80000E94B02CF5CF0895CF93C82F682F86EEF1
:103C900095E00E94DD2C90916E059C2790936E0517
:103CA000CF910895A1E0B0E0E8E5FEE10C942C2F5F
:103CB00099830E94441E9981892F0E94441E219657
:103CC000E2E00C94482F1F93CF93DF93182FEB0162
:103CD00010926E0565EB70E086EE95E00E94590645
:103CE00062E670E086EE95E00E945906812F0E9400
:103CF000441ECE010E94521EDF91CF911F91089564
:103D000060916E0586EE95E00E94DD2C0895A1E29B
:103D1000B0E0EDE8FEE10C94282F7B018A018C30A5
:103D200009F452C108F040C0863009F4BCC018F54F
:103D3000833009F491C070F4813009F472C082308C
:103D400009F049C26BE170E082E00E94631E03EA61
:103D500015E078C0843009F487C0853009F03BC293
:103D600060914D0570E0660F771F85E00E94631E2D
:103D70000EE415E086C0893009F4A7C070F48730DE
:103D800009F49BC0883009F026C261E070E088E049
:103D90000E94631E8091D80524C28A3009F4CAC0EB
:103DA0008B3009F4F1C017C28A3609F474C1D8F413
:103DB000873609F439C138F4853609F40DC18636E1
:103DC00009F41EC108C2883609F436C1893609F0E3
:103DD00002C261E070E089E60E94631E0E947A06DA
:103DE0000E94BF06F6C18D3609F4D3C138F48B3674
:103DF00009F490C18C3609F499C1EDC18E3609F4ED
:103E0000DDC1873C09F0E7C161E070E087EC0E940A
:103E1000631E81E00E94441E0E94801E10926F0566
:103E2000E4C169E270E081E00E94631E0AE715E0E8
:103E3000F80181918F010E94441EF5E0033A1F07AB
:103E4000B9F7D1C1F80181918F010E94441EF5E0BC
:103E50000E3B1F07B9F7C7C161E070E083E00E9425
:103E6000631E0E947018BDC161E070E084E00E9492
:103E7000631E81E00E94441E0E94801E0E94A316C1
:103E8000B4C180914D0590E0880F991F98012E5480
:103E900035402817390708F0A6C1F80181918F0134
:103EA0000E94441EEECF62E070E086E00E94631E36
:103EB00088E893E00E94521E96C161E070E087E0BE
:103EC0000E94631E80914C058CC186E6898361E067
:103ED000CE0101960E940D0C0E948B0B83E0809313
:103EE000770568EC70E080E090E00E94A629809160
:103EF00077058430D9F48FE70E9495090E94A809BC
:103F00008983863469F460E270E089E00E94631E70
:103F100010E20E94A8090E94441E1150D1F763C10B
:103F200061E070E089E00E94631E53C161E070E0CF
:103F300089E054C169E170E08AE00E94631E10923A
:103F4000BE05209176058091C3059091C405A0918E
:103F5000C505B091C605222311F0806801C08F7796
:103F60008093C3059093C405A093C505B093C6057F
:103F70000EEB15E0F80181918F010E94441EF5E0DF
:103F8000073D1F07B9F72FC161E270E08BE00E9487
:103F9000631E8091AA048F3F39F08091AA0491E0BA
:103FA000980F9093AA0402C08091AA040E94441E14
:103FB00010E0812F0E9430160E9427090E94521E95
:103FC0001F5F1031B1F70FC161E070E08CE00E941B
:103FD000631E8091D70505C161E070E085E60E940F
:103FE000631E89E2E816F10409F0FAC0D801EAE795
:103FF000F5E08D91819385E0E33AF807D1F7E9C0C8
:1040000061E070E086E60E94631EEBE1EE16F104CB
:1040100009F0E6C0D801E3EAF5E08D91819385E0EF
:10402000EE3BF807D1F7D5C061E070E087E60E946B
:10403000631E0E94710DCDC061E070E088E60E94B1
:10404000631E85E789838BE1E3EAF5E0DE011296E2
:1040500001900D928A95E1F76CE1CE0101960E94E4
:104060000D0C0E948B0B83E08093770560E273E078
:1040700080E090E00E94A62980917705843009F0C5
:10408000AFC08FE70E9495090E94A80989838535F2
:1040900009F0A6C09EC061E070E08AE60E94631E3F
:1040A00089E6898361E0CE0101960E940D0C0E9491
:1040B0008B0B83E08093770560E273E080E090E013
:1040C0000E94A62980917705843009F089C08FE786
:1040D0000E9495090E94A80989838E010E5F1F4FD7
:1040E0007E01EDE1EE0EF11C0E94A809F80181931A
:1040F0008F01EE15FF05C1F78BE1FE013296A3EAB1
:10410000B5E001900D928A95E1F78981893409F033
:1041100067C05FC061E070E08BE60E94631EF8013B
:1041200080818093D8050E947A0D53C061E070E0D1
:104130008CE60E94631EF0E2EF16F10461F487E65C
:10414000898380E2F801DE01129601900D928A9532
:10415000E1F761E203C087E4898361E0CE01019663
:104160000E940D0C0E948B0B83E0809377056CE41A
:1041700074E080E090E00E94A62980917705843069
:1041800079F58FE70E9495090E94A809873441F5C7
:1041900020C061E070E08DE60E94631E89E1E816B0
:1041A000F104F1F4D801EEEBF5E08D91819385E017
:1041B000E73DF807D1F70E94BA130BC061E070E049
:1041C0008EE60E94631EF80180818093D7050E94CD
:1041D0005B0D81E006C061E070E08AEC0E94631E26
:1041E00080E00E94441E0E94801EA196E6E00C948E
:1041F000442FA0E0B0E0EFEFF0E20C94262FCAECE1
:10420000D3E014E606E035E0F32E44E0E42E53E07C
:10421000D52E62E0C62E86EE95E00E94832C892B77
:1042200009F49BC086EE95E00E94B02C282F809365
:1042300035044091340450E04730510560F7FA01ED
:10424000EE52FF4F0C94532F853B29F781E080936A
:104250003404E1CF823609F07DC0C0923404DBCF54
:104260008093330480933204D0923404D4CF9C01E1
:1042700033273093310420933004909132049827EF
:1042800090933204E0923404C6CF382F2227409115
:10429000300450913104242B352B3093310420937A
:1042A000300490913204982790933204F0923404B1
:1042B0002536310508F4AFCF61E070E08CEC0E9448
:1042C000631E81E00E94441E0E94801E43C0209114
:1042D0002E0430912F04F901E653FC4F8083909116
:1042E0003204982790933204C901019690932F04C9
:1042F00080932E042091300430913104821793076B
:1043000008F489CF0093340486CF8091320482135D
:104310000BC060912E0470912F044AEC53E0809101
:1043200033040E94871E0DC062E070E08BEC0E9497
:10433000631E809133040E94441E80916E050E948A
:10434000441EFE01812F11928A95E9F710922F04E5
:1043500010922E04109234045ECFCDB7DEB7E8E0A1
:104360000C94422F81E080936F0580916F05882324
:1043700049F086EE95E00E94832C892BB1F30E94D0
:10438000F920F3CF0895AAE2B0E0E9ECF1E20C9451
:10439000242F0E9477296B017C0181E00E949C0AF6
:1043A00086EE95E00E94832C892B29F086EE95E01D
:1043B0000E94B02CF5CF5E9811E072E6B72EE9E2CC
:1043C000AE2E03E00E9477296C197D098E099F09A2
:1043D000693C710581059105D0F11123C1F10E945D
:1043E00077296B017C015D9A80ED97E00E94AE0712
:1043F000B982EAE7F5E0DE0112968A2D01900D926E
:104400008A95E1F76AE2CE0101960E940D0C5D9853
:1044100080E090E00E94AE07009377050E948B0B2E
:1044200062E370E080E090E00E94A6298091770529
:10443000843061F4009377058FE70E9495090E940C
:10444000A80911E0823419F410E001C011E08EE0F7
:104450000E949C2A892B81F411E00EC05E9A5D9A1D
:1044600086EE95E00E94B02C8D309105A9F05CF4A9
:104470000A9791F05E985D9886EE95E00E94832CF5
:10448000892B61F79FCF8332910579F082349105B2
:1044900089F70E94B221EECF62EB71E086EE95E0E3
:1044A0000E945D2B0E941A1EE5CF0E94A316E2CF48
:1044B0008F929F92AF92BF92CF92DF92EF92FF9234
:1044C0001F93CF93DF938EE00E949C2A892B09F0E3
:1044D00089C068EC70E080E090E00E94A62980E04E
:1044E00090E00E94AE070E9477294B015C016B01AE
:1044F0007C0180ECC80E82E1D81EE11CF11C0E94F8
:1045000077296C157D058E059F0530F48EE00E949D
:104510009C2A892BA1F364C08EE00E949C2A892BDF
:1045200009F05EC080ED97E00E94AE070E947729F7
:104530006B017C01D0E0C1E088E4880E86E2981E21
:10454000A11CB11C11E08EE00E949C2A892B21F550
:104550008C149D04AE04BF0430F480ED97E00E94FB
:10456000AE07D1E0F0CF0E9477296C197D098E0942
:104570009F09693C71058105910528F30E947729FF
:104580006B017C01C12719F080ED97E002C080E04B
:1045900090E00E94AE07D7CF80E090E00E94AE0787
:1045A000DD23B9F08091D70590E0019665E070E0D9
:1045B0000E94C72E8093D7050E945B0D0E94D513E1
:1045C0000E947A0D64EF71E080E090E00E94A629DD
:1045D00009C080E00E94DF060E94F2110E94710D66
:1045E0000E94C321DF91CF911F91FF90EF90DF9048
:1045F000CF90BF90AF909F908F900895CF92DF9211
:10460000EF92FF9280E00E94F8070E94CF0761E0DE
:1046100089E00E94302A60E089E00E94692A61E016
:1046200086E00E94302A61E085E00E94302A60E046
:104630008EE00E94302A60E08FE00E94302A61E024
:104640008FE00E94692A60E080E10E94302A61E0E8
:1046500080E10E94692A60E088E00E94302A61E0DF
:1046600088E00E94692A61E081E10E94302A60E0CE
:1046700081E10E94692A0E949F0740E052EC61E0BC
:1046800070E086EE95E00E94CB2D0E94D5130E942B
:104690007A0D0E94BA138FEF8093AA040E94E40758
:1046A00078940E9477296B017C018091AA048F3F46
:1046B00059F40E9477296C197D098E099F09603D84
:1046C00077408105910588F380ED97E00E94AE0761
:1046D00061E08EE00E94692A5E9A86EE95E00E9473
:1046E000832C892B29F086EE95E00E94B02CF5CF23
:1046F0006DEF72E086EE95E00E943E2B88E893E035
:104700000E94620C64E173E086EE95E00E943E2B0D
:104710004AE050E064E070E086EE95E00E940E2CE6
:1047200062E370E080E090E00E94A62986EE95E0CA
:104730000E94832C04970CF186EE95E00E94B02C29
:1047400082349105D1F486EE95E00E94B02C8E342F
:10475000910599F486EE95E00E94B02C8434910581
:1047600061F486EE95E00E94B02C819731F480E0F0
:1047700090E00E94AE070E94C32140917B055091BA
:104780007C0560917D0570917E05DB01CA01019772
:10479000A109B1090497A105B10568F44093A904E2
:1047A000433029F440EA56E861E070E004C040E09C
:1047B00052EC61E070E086EE95E00E94CB2D0E9405
:1047C00058225E9880E090E00E94AE070E94BA13E3
:1047D0001092C9048091C30583FF11C080918F0599
:1047E000882351F080919605882331F080919D05B2
:1047F000882311F087E001C085E08093C90480E040
:104800000E949C0A8091CA040E94D0090E948B0BCE
:1048100010923F0410923E0410923D04F12C8091BE
:10482000D8058F15B0F062E370E080E090E00E9460
:10483000A62980ED97E00E94AE0762E370E080E079
:1048400090E00E94A62980E090E00E94AE07F394D9
:10485000E6CF8091A20584FF08C0982F987181E06F
:10486000983109F080E00E94AE118FE00E94F807B5
:10487000FF90EF90DF90CF900895EF92FF920F930B
:104880001F93CF93DF938C016EE770E086EE95E087
:104890000E945906E801F12CF0E2EF2E8E0188818A
:1048A0008D57823048F46DE770E086EE95E00E9407
:1048B000590688818E2588832196F801608186EECD
:1048C00095E00E94DD2CF394F9E0FF12E7CF6EE74C
:1048D00070E086EE95E00E945906CDB7DEB7E6E0BF
:1048E0000C94442FA9E0B0E0E8E7F4E20C942C2FFC
:1048F0009091CB0491110EC09EEF99838A836B83B4
:1049000050E0559547954C832D83198618861F8254
:104910001E822EC04091D004842F90E0B4E0959583
:104920008795BA95E1F7242F2F7030E0821793070F
:1049300019F18DEF89831B82FE01349650E0842F9C
:1049400090E0A4E095958795AA95E1F7242F2F7024
:1049500030E08217930749F0DC01AF52BB4F8C91D6
:104960008193405F5F5F563051F74093D0045A8384
:10497000CE0101960E943D248091CB0490E00196E7
:1049800066E070E00E94C72E8093CB042996E2E097
:104990000C94482FA0E0B0E0E0EDF4E20C94252F59
:1049A0006C016EE770E086EE95E00E945906860184
:1049B000E12CF12CC0E0D0E030E2B32EF8016081B0
:1049C00083E8860F823078F46DE770E086EE95E03C
:1049D0000E945906F80160816B2570E086EE95E033
:1049E0000E94590604C086EE95E00E94DD2CE11479
:1049F000F10459F0F80180819E01280F311DC90191
:104A0000C92FDD27C80FD91FDD273FEFE31AF30AAF
:104A100089E0E816F10459F028E0E216F10421F4E7
:104A20008C2F8095F60180870F5F1F4FC7CFCDB7C2
:104A3000DEB7E9E00C94412FA9E0B0E0E2E2F5E254
:104A40000C942C2FE82F362F8091CB0490E0019608
:104A500064E270E00E94C72E8093CB0458E959832A
:104A600050E15A83813089F048F08230B9F08330C8
:104A7000D9F48B8381EF8C833D8319C085E08B83D0
:104A800081EF8C832F5F2D8312C08B8381EF8C830A
:104A900084E6489FA00111245D8309C084E08B83D4
:104AA00081EF8C83ED8303C00E94EB1104C0CE0123
:104AB00001960E94CA242996E2E00C94482FA2E0B5
:104AC000B0E0E5E6F5E20C94212F182F762E2A832C
:104AD00049830E9483296B017C018091E1048090CD
:104AE000CC049090CD04A090CE04B090CF042A8145
:104AF00049818823C1F0D701C60188199909AA09FB
:104B0000BB094C015D0191EE89169EE29906A10454
:104B1000B10420F1241708F4422F202F672D812F94
:104B20000E941C2513C0D701C60188199909AA093A
:104B3000BB094C015D0191E3891695E79906A10433
:104B4000B10460F0672D812F0E947224C092CC04C2
:104B5000D092CD04E092CE04F092CF042296EDE004
:104B60000C943D2FA2E2B0E0E8EBF5E20C94222F8A
:104B70008CE00E94B70981110DC06CE173E086EEF4
:104B800095E00E946F2B5E9A80E00E949C0A0E9432
:104B90008B0B5E9886EE95E00E94832C892B01F1A9
:104BA00086EE95E00E94B02C9091A904992319F00B
:104BB0000E941114EFCF40913E0450E09A012F5F04
:104BC0003F4F2F71332760913F0470E0261737075E
:104BD00009F3FA01E75BFB4F808320933E04DACFB1
:104BE00080917705843009F086C00E948329611581
:104BF00071058105910549F06093BB047093BC0475
:104C00008093BD049093BE040CC081E090E0A0E0CE
:104C1000B0E08093BB049093BC04A093BD04B09318
:104C2000BE048091AD049091AE0481609093AE0477
:104C30008093AD0483E0809377058FE70E94950908
:104C400009E614E00E94A809F80181938F01F4E0BD
:104C500002371F07B9F72091720480916904982FD9
:104C6000922796FF3BC090E4922790937204982F6E
:104C700098739833F1F410E0212F30E080916904AB
:104C8000877090E0821793074CF11F5F2091A20577
:104C9000812F90E0FC01E759FB4F24FF04C0808185
:104CA0000E94CD11E9CF608186EE95E00E94DD2C57
:104CB000E3CF8F7399F480916A048093B604809156
:104CC0006B048093B40480916C048093B30480914E
:104CD0006F0490E09093AC048093AB0480913D040A
:104CE000813019F482E080933D0480913D0483304B
:104CF00011F410923D040E9483296B017C01809184
:104D0000AF049091B004A091B104B091B2040097A7
:104D1000A105B105C9F0A7019601281B390B4A0B63
:104D20005B0BDA01C901883B9B40A105B10560F02E
:104D30000E94E6098093B5041092AF041092B0046B
:104D40001092B1041092B2048091BF049091C004FB
:104D5000A091C104B091C20446015701881A990A72
:104D6000AA0ABB0A8AE795E00E94120886169706EF
:104D7000A806B90608F4B1C0C092BF04D092C0041E
:104D8000E092C104F092C2040E9457068091AA04E6
:104D90008830A0F08091C3059091C405A091C5050D
:104DA000B091C6055CE1B695A795979587955A95FC
:104DB000D1F7892B8A2B8B2B09F0C4C18091AA04CF
:104DC0008F5F8093AA048091BB049091BC04A09152
:104DD000BD04B091BE040097A105B105F1F0C81A59
:104DE000D90AEA0AFB0A8AE795E00E9412086C15C4
:104DF0007D058E059F0508F01BC18091C30584FDCC
:104E000004C080ED97E00E94AE071092BB041092A0
:104E1000BC041092BD041092BE0490917204907C68
:104E20009093720450913E0480913F0420913D0480
:104E3000581709F41AC1223009F017C190589093FD
:104E40007204E091A205E770F0E0E658FC4F608143
:104E5000693008F0F2C0615040E04613F0C0809322
:104E60003F0487E3840F90917204892B809372042E
:104E70004093400483E080933D045D9A1091870540
:104E80008091C90481113EC18091C30582FD46C154
:104E9000812F0E94970A8091CA040E94D009E09154
:104EA000A205E770F0E0E658FC4F608182E794E0ED
:104EB0000E94C60B8091C30582FD39C1E091CA04EE
:104EC000EF5FE093CA04E83109F439C1F0E0E65835
:104ED000FA4F8785882309F432C10E94350C81304E
:104EE00069F58091A205887149F18091AD04909196
:104EF000AE04880F991F9093AE048093AD0483E0B5
:104F0000809377050E948B0B0E9483296093AF04E6
:104F10007093B0048093B1049093B204672B682B14
:104F2000692B61F481E090E0A0E0B0E08093AF04F1
:104F30009093B004A093B104B093B2048091A20501
:104F400084FF2BC08091BB049091BC04A091BD0450
:104F5000B091BE04892B8A2B8B2BF9F08091AD0484
:104F60009091AE048E7F0E944809182F6091AB0487
:104F70008091B6040E940714482F612F8091B504D8
:104F800049A30E9407140091D805282F49A16091D8
:104F9000B3048091B4040E945F255D988091C7049A
:104FA0008130C1F018F08230B1F1D9C08EE00E949A
:104FB0009C2A892B09F0D3C081E08093C7040E940A
:104FC00077296093C3047093C4048093C5049093BD
:104FD000C604C5C08EE00E949C2A892B31F50E9430
:104FE0007729C090C304D090C404E090C504F09029
:104FF000C6046C197D098E099F09693E73408105BD
:10500000910508F4ACC082E08093C70480ED97E07E
:105010000E94AE07A4C08EE00E949C2A892B09F44E
:105020009EC080E090E00E94AE071092C70497C037
:1050300080E090E00E94AE07F0CE68E00DCF8517CB
:1050400009F40DCF4F5F242F30E090E0F901EE58C6
:10505000FB4FDC01A75BBB4F7C917083F901E05CE7
:10506000FB4F708301968F71F8CE2430B1F42091FC
:10507000400481E494E0A3E7B4E0FC013E2F381B38
:10508000321718F431913D93F9CF87E3820F909155
:105090007204892B80937204EDCE8091C704823014
:1050A00051F49160909372045E9A8E010F5F1F4FCE
:1050B000F12CB80110C05E9880913D04811103C0AD
:1050C00081E080933D0480913D04833071F784E05A
:1050D00080933D04EACF8F2D69A37AA30E943016F6
:1050E000F801819391938F01F39469A17AA1F0E182
:1050F000FF12F1CF8091A20543E754E087700E9430
:105100009708BBCE112309F4BFCE9091C80421E0CB
:10511000290F2093C8049813B7CE1DC08FE00E94BA
:105120009C2A892B09F0B4CE5E9A17E0B1CE8FE0AD
:105130000E949C2A892B09F0C1CE5E98BFCE1092A6
:10514000CA04CBCE8091AA04883009F45E9A89E023
:105150008093AA04C2CE1092C804115095CEA29694
:10516000ECE00C943E2F8230E8F4E82FF0E0EE0FF4
:10517000FF1FE752FA4F71836083813041F08091C5
:1051800069008C7F842B80936900E89A0895809150
:105190006900440F551F440F551F837F842B809354
:1051A0006900E99A08951F920F920FB60F92112489
:1051B0002F933F934F935F936F937F938F939F931F
:1051C000AF93BF93EF93FF938091D9059091DA0548
:1051D000892B29F0E091D905F091DA050995FF9125
:1051E000EF91BF91AF919F918F917F916F915F915F
:1051F0004F913F912F910F900FBE0F901F901895D8
:105200001F920F920FB60F9211242F933F934F933B
:105210005F936F937F938F939F93AF93BF93EF931E
:10522000FF938091DB059091DC05892B29F0E091BB
:10523000DB05F091DC050995FF91EF91BF91AF91EE
:105240009F918F917F916F915F914F913F912F919E
:105250000F900FBE0F901F9018951F920F920FB6D0
:105260000F9211242F933F938F939F93AF93BF93EC
:105270008091DE059091DF05A091E005B091E105F8
:105280003091DD0523E0230F2D3720F40196A11D79
:10529000B11D05C026E8230F0296A11DB11D209364
:1052A000DD058093DE059093DF05A093E005B093C4
:1052B000E1058091E2059091E305A091E405B091AC
:1052C000E5050196A11DB11D8093E2059093E305CC
:1052D000A093E405B093E505BF91AF919F918F91A5
:1052E0003F912F910F900FBE0F901F9018952FB7E1
:1052F000F8946091DE057091DF058091E005909152
:10530000E1052FBF08953FB7F8948091E205909191
:10531000E305A091E405B091E50526B5A89B05C07D
:105320002F3F19F00196A11DB11D3FBF6627782FB1
:10533000892F9A2F620F711D811D911D42E0660F0A
:10534000771F881F991F4A95D1F70895CF92DF9252
:10535000EF92FF92CF93DF936B017C010E94832930
:10536000EB01C114D104E104F10479F00E94832916
:105370006C1B7D0B683E7340A0F381E0C81AD10816
:10538000E108F108C851DC4FECCFDF91CF91FF90DD
:10539000EF90DF90CF900895789484B5826084BDBB
:1053A00084B5816084BD85B5826085BD85B5816029
:1053B00085BDEEE6F0E0808181608083E1E8F0E089
:1053C0001082808182608083808181608083E0E8B8
:1053D000F0E0808181608083E1EBF0E08081846097
:1053E0008083E0EBF0E0808181608083EAE7F0E099
:1053F00080818460808380818260808380818160FD
:1054000080838081806880831092C10008958330FA
:1054100081F028F4813099F08230A1F0089586302F
:10542000A9F08730B9F08430D1F4809180008F7D6D
:1054300003C0809180008F7780938000089584B5A9
:105440008F7702C084B58F7D84BD08958091B000B0
:105450008F7703C08091B0008F7D8093B000089556
:10546000CF93DF9390E0FC01ED50F44F2491FC01C9
:10547000E95FF34F8491882349F190E0880F991FE9
:10548000FC01E15DF34FA591B4918B5D934FFC015D
:10549000C591D4919FB7611108C0F8948C91209563
:1054A00082238C93888182230AC0623051F4F8945D
:1054B0008C91322F309583238C938881822B888323
:1054C00004C0F8948C91822B8C939FBFDF91CF9175
:1054D0000895A1E0B0E0EFE6FAE20C942A2F282F1D
:1054E00030E0F901E152F44F8491F901ED50F44FAD
:1054F0001491F901E95FF34F04910023C9F0882367
:1055000021F069830E94072A6981E02FF0E0EE0F05
:10551000FF1FEB5DF34FA591B4919FB7F8948C9169
:10552000611103C01095812301C0812B8C939FBF13
:105530002196E4E00C94462FCF93DF93282F30E0A0
:10554000F901E152F44F8491F901ED50F44FD491F7
:10555000F901E95FF34FC491CC2391F081110E94CE
:10556000072AEC2FF0E0EE0FFF1FE55EF34FA59149
:10557000B4912C912D2381E090E021F480E002C0D1
:1055800080E090E0DF91CF9108958E3008F08E504A
:10559000877020919D0190E4299F90011124822B16
:1055A00080937C0080917A00806480937A0080915F
:1055B0007A0086FDFCCF809178002091790090E000
:1055C000922B0895A0E0B0E0E8EEFAE20C94262FCA
:1055D0006C017A01EB01E60EF71E00E010E0CE153B
:1055E000DF0561F06991D601ED91FC910190F081A8
:1055F000E02DC6010995080F191FF1CFC801CDB7DD
:10560000DEB7E8E00C94422F6115710589F0DB01EB
:105610000D900020E9F7AD0141505109461B570B91
:10562000DC01ED91FC910280F381E02D0995089554
:1056300080E090E00895EF92FF920F931F93CF9335
:10564000DF938C01FB01C0E0D0E064917F018FEF1C
:10565000E81AF80A662361F0D801ED91FC910190F7
:10566000F081E02DC8010995C80FD91FF701EDCFD2
:10567000CE01CDB7DEB7E6E00C94442F0E94042B98
:105680000895DC01ED91FC910190F081E02D0995E8
:1056900008950F931F93CF93DF93EC016DE00E9469
:1056A000412B8C016AE0CE010E94412B800F911F9B
:1056B000DF91CF911F910F9108950F931F93CF9377
:1056C000DF93EC010E941B2B8C01CE010E94492B21
:1056D000800F911FDF91CF911F910F9108950F932C
:1056E0001F93CF93DF93EC010E94042B8C01CE011A
:1056F0000E94492B800F911FDF91CF911F910F9135
:1057000008950F931F93CF93DF93EC010E94412BD9
:105710008C01CE010E94492B800F911FDF91CF9108
:105720001F910F910895A1E2B0E0E9E9FBE20C942A
:10573000222F7C01C42EE52FCB01D22E19A221E00D
:105740002D1510F02AE0D22E8E010F5D1F4F8D2CEB
:10575000912CA12CB12C6C2D7E2FA50194010E94BF
:10576000DB2E8C2DD29E80191124015011098A3014
:1057700010F4805D01C0895CF8018083211531053A
:105780004105510521F0C22EE32FCA01E4CFB80133
:10579000C7010E94042BA196ECE00C943E2FA0E0E0
:1057A000B0E0E5EDFBE20C94262FEC016A017B01F1
:1057B0002115310541F4E881F9810190F081E02D56
:1057C000642F09951DC02A303105A9F477FF12C056
:1057D0006DE20E94412B8C0144275527BA014C19D8
:1057E0005D096E097F092AE0CE010E94932B800F8C
:1057F000911F06C02AE0B701A601CE010E94932B9B
:10580000CDB7DEB7E8E00C94422F9A01AB016627D2
:1058100057FD6095762F0E94CF2B08950F931F930D
:10582000CF93DF93EC019A01AB01662757FD60959A
:10583000762F0E94CF2B8C01CE010E94492B800F26
:10584000911FDF91CF911F910F910895211531057F
:1058500049F4DC01ED91FC910190F081E02D642F81
:10586000099508950E94932B08959A01462F50E0C0
:1058700060E070E00E94262C08959A01AB0160E080
:1058800070E00E94262C08950F931F93CF93DF930F
:10589000EC010E94262C8C01CE010E94492B800F26
:1058A000911FDF91CF911F910F9108950F931F9337
:1058B000CF93DF93EC019A01AB0160E070E00E94AE
:1058C000262C8C01CE010E94492B800F911FDF9165
:1058D000CF911F910F9108950F931F93CF93DF9353
:1058E000EC019A01462F50E060E070E00E94262C07
:1058F0008C01CE010E94492B800F911FDF91CF9127
:105900001F910F910895FC0124853585F901E05C14
:10591000FF4F80819181F901EE5BFF4F2081318142
:10592000821B930B8F7399270895FC0184859585BD
:10593000FC01E05CFF4F40815181FC01EE5BFF4FB9
:10594000208131814217530741F00190F081E02D11
:10595000E80FF91F808190E008958FEF9FEF089581
:10596000FC0184859585FC01E05CFF4F40815181FD
:10597000FC01EE5BFF4F208131814217530779F024
:10598000A081B181A80FB91F8C91208131812F5F37
:105990003F4F2F7333273183208390E008958FEF9B
:1059A0009FEF0895FC0181A1882329F0A489B5897E
:1059B0008C9186FFFBCF11A20895CF93DF93FC015A
:1059C00026853785D901A05CBF4F8D919C91119799
:1059D00001968F739927E901CE5BDF4F488159818A
:1059E00084179507D9F30D90BC91A02DA20FB31F7A
:1059F0006C93A685B785A05CBF4F11969C938E9340
:105A0000A689B7892C9181E090E0078C02C0880FAD
:105A1000991F0A94E2F7282B2C9381E081A3048834
:105A2000F589E02D80818064808381E090E0DF91C2
:105A3000CF91089508951F920F920FB60F921124DF
:105A40002F933F934F938F939F93EF93FF93809167
:105A5000C00082FD1CC04091C60080918C069091D0
:105A60008D0601968F73992720918E0630918F06AF
:105A70008217930771F0E0918C06F0918D06E45B3C
:105A8000F94F408390938D0680938C0602C08091DD
:105A9000C600FF91EF919F918F914F913F912F9170
:105AA0000F900FBE0F901F90189586EE95E00E9404
:105AB000832C892B11F00E941A2D08951F920F92AA
:105AC0000FB60F9211242F933F938F939F93EF93D1
:105AD000FF93209148063091490680914A069091A3
:105AE0004B062817390731F48091C1008F7D8093D0
:105AF000C10014C0E0914A06F0914B06E85FF94FEF
:105B0000208180914A0690914B0601968F739927C8
:105B100090934B0680934A062093C600FF91EF9125
:105B20009F918F913F912F910F900FBE0F901F90DB
:105B30001895A0E0B0E0EFE9FDE20C94222FFC0103
:105B40001382128288EE93E0A0E0B0E08483958314
:105B5000A683B7838CEB93E09183808375876487FA
:105B600057874687318B208B138B028BF58AE48A0B
:105B7000D78AC68AB18EA08E938E828E8F85848FAF
:105B80008889858F8989868F8A89878F8B8980A369
:105B9000ECE00C943E2FCF92DF92EF92FF92CF93E6
:105BA000DF93EC016A017B01411581EE5807610525
:105BB0007105F9F0EC89FD8981E090E008A002C050
:105BC000880F991F0A94E2F7808360E079E08DE303
:105BD00090E0A70196010E94DB2E21503109410976
:105BE00051095695479537952795211580E1380736
:105BF00098F0EC89FD89108260E874E88EE190E00D
:105C0000A70196010E94DB2E21503109410951095B
:105C10005695479537952795E889F9893083EA891C
:105C2000FB89208319A2EE89FF89408181E090E001
:105C30009C010C8C02C0220F331F0A94E2F7422B06
:105C40004083EE89FF8940819C010D8C02C0220FA8
:105C5000331F0A94E2F7422B4083EE89FF8940818B
:105C60009C010E8C02C0220F331F0A94E2F7422BD4
:105C70004083EE89FF8920810F8C02C0880F991F15
:105C80000A94E2F7809582238083DF91CF91FF9081
:105C9000EF90DF90CF9008958F929F92AF92BF9236
:105CA000CF92DF92EF92FF920F931F9381E08F9339
:105CB00085E08F9387E08F9383E08F9384E08F93C9
:105CC000E6EC8E2E912CF2ECAF2EB12CA1ECCA2E6C
:105CD000D12CB0ECEB2EF12C04EC10E025EC30E0F4
:105CE00048E056E06CE476E086EE95E00E94992D5F
:105CF0000F900F900F900F900F901F910F91FF90AA
:105D0000EF90DF90CF90BF90AF909F908F900895CD
:105D10000E94CC290E94FE22C5E5DDE20E94B22548
:105D20002097E1F30E94552DF9CFA29FB001B39FB8
:105D3000C001A39F700D811D1124911DB29F700D94
:105D4000811D1124911D08950E94952EA59F900DEF
:105D5000B49F900DA49F800D911D11240895B7FF4D
:105D60000C94A42E0E94A42E821B930B0895DB0199
:105D70008F939F930E94A42EBF91AF91A29F800DFD
:105D8000911DA39F900DB29F900D1124089597FB34
:105D9000072E16F4009407D077FD09D00E94592FE2
:105DA00007FC05D03EF4909581959F4F089570951E
:105DB00061957F4F0895A1E21A2EAA1BBB1BFD011E
:105DC0000DC0AA1FBB1FEE1FFF1FA217B307E407DA
:105DD000F50720F0A21BB30BE40BF50B661F771F32
:105DE000881F991F1A9469F7609570958095909512
:105DF0009B01AC01BD01CF010895052E97FB1EF458
:105E000000940E94142F57FD07D00E94DB2E07FC40
:105E100003D04EF40C94142F509540953095219555
:105E20003F4F4F4F5F4F08959095809570956195C6
:105E30007F4F8F4F9F4F08952F923F924F925F92C7
:105E40006F927F928F929F92AF92BF92CF92DF928A
:105E5000EF92FF920F931F93CF93DF93CDB7DEB7EF
:105E6000CA1BDB0B0FB6F894DEBF0FBECDBF099483
:105E70002A88398848885F846E847D848C849B84DA
:105E8000AA84B984C884DF80EE80FD800C811B81E8
:105E9000AA81B981CE0FD11D0FB6F894DEBF0FBE17
:105EA000CDBFED010895EE0FFF1F0590F491E02D99
:105EB0000994AA1BBB1B51E107C0AA1FBB1FA61751
:105EC000B70710F0A61BB70B881F991F5A95A9F7A3
:105ED00080959095BC01CD0108958F929F92AF92CD
:105EE000BF92CF92DF92EF92FF92CF93DF93EC01BC
:105EF000688179818A819B81611571058105910590
:105F000021F464E279ED8BE597E02DE133EF41E098
:105F100050E00E94FD2E49015A019B01AC01A7EA05
:105F2000B1E40E94A42E6B017C01ACEEB4EFA5019C
:105F300094010E94B22EC60ED71EE81EF91EF7FE6F
:105F400006C081E0C81AD108E10880E8F80AC882D2
:105F5000D982EA82FB82C701B6019F77DF91CF9198
:105F6000FF90EF90DF90CF90BF90AF909F908F9079
:105F700008950E946D2F089586E091E00E946D2F94
:105F80000895609306017093070180930801909330
:105F9000090108952F923F925F926F927F928F92A4
:105FA0009F92AF92BF92CF92DF92EF92FF920F93A8
:105FB0001F93CF93DF938B01EA016115710521F0E7
:105FC000DB018C9311969C93209739F09E0122500F
:105FD00031092332310508F0D8C07C016701BFEFD9
:105FE000CB1ADB0A5601F7016080862D90E00E94F3
:105FF000FC30892B11F07601F1CFFDE26F120AC05F
:10600000570182E0A80EB11CD70111966C9077243D
:1060100073940BC0BBE26B1207C05701E2E0AE0EF7
:10602000B11CD70111966C90712CCE018F7E892BFB
:1060300089F4B0E36B1237C0F50180818F7D88351C
:10604000D1F46180F2E0AF0EB11C872D8260782E12
:10605000C0E1D0E0CA30D10551F1C031D10521F005
:10606000C830D10599F409C0CC24CA94DC2CEC2C9E
:10607000AFE0FA2E22C0209769F7C8E0D0E0CC2428
:10608000CA94DC2CEC2CFFE1FF2E17C06FEF7FEFE2
:10609000CB019E01442737FD4095542F0E94DB2EF3
:1060A00069017A010AC02097A9F6CAE0D0E0E9E9BF
:1060B000CE2EDC2CEC2CE9E1FE2EF50160E020E098
:1060C00030E0A9014E01AA2497FCA094BA2C1F012C
:1060D00070ED572E560CA9E0A51570F48FEB860DC8
:1060E0008A3118F499EC592E06C08FE9860D8A3151
:1060F00048F589EA582E560C852D90E08C179D079F
:106100000CF56F3FD9F0C216D306E406F50698F0F9
:10611000C501B4010E94B72E9B01AC01852D90E012
:10612000A0E0B0E0280F391F4A1F5B1F281739076E
:106130004A075B0710F46FEF01C061E03196D101AF
:106140006C90C5CF0115110551F0662311F0319700
:1061500003C071FE04C03297D801ED93FC9370FE2A
:1061600007C050954095309521953F4F4F4F5F4F59
:1061700067FF10C082E290E09093910680939006B2
:106180006FEF7FEF8FEF9FEF07C060E070E080E080
:1061900090E002C0B901CA01DF91CF911F910F9128
:1061A000FF90EF90DF90CF90BF90AF909F908F9037
:1061B0007F906F905F903F902F900895FC0188270B
:1061C0009927E89421912032E9F3293010F02E30FC
:1061D000C8F32B3241F02D3239F4689404C00E9488
:1061E0003031820F911D219120532A30C0F31EF4CB
:1061F000909581959F4F0895911150C0803219F06C
:1062000089508550D0F7089548EC53E00E94093139
:106210000895FA01A191B081009719F41097E1F067
:10622000CD01DC01CD010D90002011F4C00113C09F
:10623000FB012191222319F02015D9F7F3CFFB019F
:106240002191201519F41E92119606C02223C1F740
:106250000D900020A1F7D001FA01A193B083089519
:106260007AE0979F902D879F802D910D112408959E
:10627000F999FECF92BD81BDF89A992780B508950E
:10628000262FF999FECF1FBA92BD81BD20BD0FB652
:10629000F894FA9AF99A0FBE0196089599278827DB
:0662A0000895F894FFCF01
:1062A60000009206200001000000FF00020002002C
:1062B60002000200020002000200020002000200C8
:1062C6000200020002000200020002802500000512
:1062D600400AA1204EA50020244EA52C2330C01232
:1062E60000001A400AA1204EA5001B1E27522C238F
:1062F600308025000005400AA1204EA50020244E2E
:10630600A52C2330004B000006400AD0009D490012
:106316007B289D492C233000E1000005400A4501F9
:10632600D7DC03B81E0EBF00232E48E801008A40C2
:106336000A6001555502AD1E20000023C8015458BD
:106346002074696D656F75742100596573004E6F11
:10635600002C00386368004E2F41002C205B005D46
:106366002028002900486F70206368616E6E656C96
:10637600200020402000456E746572696E672061BA
:1063860064617074697665206368616E6E656C2001
:1063960073656C656374696F6E2C207069636B69D5
:1063A6006E673A007363616E6E6572206D6F646529
:1063B600004E4F5420454E41424C45440053656EB5
:1063C60064696E672073657474696E677320746F91
:1063D6002052580A00526573657474696E6720739B
:1063E600657474696E6773206F6E2052580A004197
:1063F600626F727465642065646974730A00696EFD
:1064060076616C69642073656C656374696F6E0090
:106416000D0A496E76616C696420696E7075742028
:106426002D20646973636172646564210700536596
:106436007474696E677320736176656420746F2067
:10644600454550524F4D0A00526576657274656433
:106456002073657474696E67732066726F6D20456C
:106466004550524F4D0A004C6F6164656420666169
:1064760063746F72792064656661756C74730A0063
:106486004B657920616E64206368616E6E656C731E
:106496002072616E646F6D697A65640A004F70657B
:1064A6006E4C52536E67205458207374617274692F
:1064B6006E672000206F6E20485720006D6F647550
:1064C6006C65206C6F636B65643F00342B34003859
:1064D60000382B340031320031322B340031360093
:1064E60050504D0052535349005344410053434CBE
:1064F60000525844005458440041494E004C42450D
:1065060045500053504B54524D005342555300537F
:10651600554D44004C4C494E440000070B0C1011DD
:106526001500B7012B032F033103350338033D0351
:10653600B7014003440349034D035103550359036F
:106546005D0363036A036F0374038D028D028D027C
:106556008D02160A1322312900000000DD2CE22AE2
:08656600832CB02C952CD22CE3
:107E00000F92CDB7DEB7112484B714BE81FFF1D035
:107E100082E08093C00088E18093C10086E0809377
:107E2000C20080E18093C4008EE0CDD088249924E4
:107E3000CC24C394F5E0DF2EE1E1EE2E73E0F72EC3
:107E4000B6D0082F813479F4B2D08983C2D0898129
:107E5000823811F481E005C0813811F485E001C059
:107E600083E09ED09AC0823411F484E103C085344B
:107E700019F485E0B6D091C0853561F498D0082F0B
:107E800010E095D090E0982E8824802A912A880CC2
:107E9000991C82C0863521F484E0A3D080E0E1CF34
:107EA000843609F04CC083D082D0A82E80D0B82E62
:107EB00000E011E07CD0F80181938F01AE16D1F77C
:107EC00088D0FB2DF53489F4E0E0F1E00BC0F9999E
:107ED000FECF92BC81BC0894811C911C819180BD15
:107EE000FA9AF99AEA1598F358C08B2D863409F05E
:107EF00054C0F401F7BEE89507B600FCFDCFF401CD
:107F0000A0E0B1E02C9130E011968C91119790E0B7
:107F1000982F8827822B932B12960C01C7BEE895C9
:107F20001124329681E0A038B80761F7F401D7BE7A
:107F3000E89507B600FCFDCFE7BEE8952EC0843774
:107F4000F1F435D034D0182F32D0B82E42D0FB2DDA
:107F5000F63421F4F40105914F010CC0FB2DF534EA
:107F600049F4F999FECF92BC81BC0894811C911C04
:107F7000F89A00B5802F14D0115049F70EC08537FC
:107F800039F427D08EE10CD085E90AD08FE069CF93
:107F9000813511F488E017D01CD080E101D050CF9A
:107FA0009091C00095FFFCCF8093C600089580910A
:107FB000C00087FFFCCF8091C00084FD01C0A89560
:107FC0008091C6000895E0E6F0E098E19083808318
:107FD0000895EDDF803219F088E0F5DFFFCF84E10E
:107FE000DFCF1F93182FE3DF1150E9F7F2DF1F9166
:0E7FF0000895282E80E0E7DFEE27FF27099492
:027FFE0001057B
:0400000300007E007B
:00000001FF
